:100000000C94E5030C942C040C942C040C942C04F8
:100010000C942C040C942C040C942C040C942C04A0
:100020000C942C040C942C040C947B100C943F1610
:100030000C94C92A0C942C040C942C040C942C04BD
:100040000C942C040C942C040C942C040C942C0470
:100050000C942C040C9454110C942C040C942C042B
:100060000C942C040C942C040C942C040C942C0450
:100070000C942C040C942C040C942C040C942C0440
:100080000C942C040C942C040C942C040C942C0430
:100090000C942C040C942C040C942C040C942C0420
:1000A0000C942C040C942C040C942C0405010902CF
:1000B000A10185020901A100050919012905150001
:1000C00025019505750181029501750381010501E1
:1000D000093009311581257F950275088106093897
:1000E0001581257F950175088106050C0A380215D2
:1000F00081257F950175088106C0C005010980A191
:1001000001850319012AB700150126B7009501756D
:10011000108100C0050C0901A101850419012AA064
:1001200002150126A002950175108100C005010984
:1001300006A1018506050719E029E71500250195A7
:1001400008750181020507190029EF1500250195A1
:10015000F0750181020508190129059505750191C0
:1001600002950175039101C00660FF0961A10109B3
:1001700062150026FF0095207508810209631500AD
:1001800026FF00952075089102C005010906A1010E
:10019000050719E029E71500250195087501810279
:1001A0009501750881010507190029FF150026FF33
:1001B0000095067508810005081901290595057542
:1001C000019102950175039101C00000000000003B
:1001D000000000000000000000000000000000001F
:1001E00000000000000000000000000000007E0F82
:1001F00000D4FFFFFFC700000078000000000000EF
:1002000000002A2B28000000000000000000000071
:10021000000000000029000000002C1E34202122D4
:1002200024342627252E362D3738271E1F2021223D
:10023000232425263333362E37381F0405060708B6
:10024000090A0B0C0D0E0F101112131415161718A6
:10025000191A1B1C1D2F3130232D350405060708E4
:10026000090A0B0C0D0E0F10111213141516171886
:10027000191A1B1C1D2F3130354C00DA0281FFD9B1
:10028000F1DB20A4A62EAF00A0C000A1C800AED50F
:1002900080A81FD300408D14200000000000000043
:1002A000000000000000000000000000000000004E
:1002B000000000000000000000000000000000003E
:1002C000000000061E3EFEFEFCFCFCFCFCFCFCFCF0
:1002D000FCFCFCFCFCFCFCFCFCFCFCFCFCFCFCFC5E
:1002E000FCFCFCFCFCFCFCFCFCFCFCFEFE3E1E06DC
:1002F00000000000000000000000000000000000FE
:1003000000000000000000000000000000000000ED
:1003100000000000000000000000000000000000DD
:1003200000000000000000000000000000000000CD
:1003300000000000000000000000000000000002BB
:10034000060E1E3E3EFEFEFF7F7FFFFF7F7F7F7F0C
:100350007F7F0F0F0F0F0F0F0F0F0F0F0F0F0F0FCD
:100360000F7F7F7F7F7FFFFFFF7F7FFFFEFE3E3E91
:100370001E0E060200000000000000000000000049
:10038000000000000000000000000000000000006D
:10039000000000000000000000000000000000005D
:1003A000000000000000000000000000000000004D
:1003B000000000000000000000000000000000003D
:1003C000000000E0FCFF070000F8FF1F0000000035
:1003D000000000000000000000000000000000001D
:1003E000000000000000001FFFF800000FFFFEE00B
:1003F00000000000000000000000000000000000FD
:1004000000000000000000000000000000000000EC
:1004100000000000000000000000000000000000DC
:1004200000000000000000000000000000000000CC
:1004300000000000000000000000000000000000BC
:1004400000383F3F0F0000001F1F0F00000000009A
:10045000000000000000000000000000000000009C
:100460000000000000000000071F1F000000073F01
:100470003F3000000000000000000000000000000D
:10048000000000000000000000000000000000006C
:1004900000000000000000000000FD377A585A00FC
:1004A0000004E6D6B4460200210116000000742FB5
:1004B000E5A3E001B700F45D003D88898654A0BA49
:1004C000D98FAB276724B0237736721CE2E03D67F3
:1004D0001A7977A2F86E68B05BBB323BC29B8EC0C4
:1004E00068C01B93EBFE8240B2642E3AFAF3AF452C
:1004F000CECE65E06B55038D1FE1A14636A8D852DC
:10050000C06227016802BA066B04C493972838AF0B
:1005100021F93C37FB14E6F885988FDA638F168D46
:10052000C84425B6F4770E668473D9049E6F93563B
:10053000BAECD45371F5AB4C78F727491284EBA58C
:100540001CC2A998791CC5E573C09C795F90FBA477
:10055000BB39E76D97B2E5F6D977884957366D060E
:100560000C904B0631D31FD45A626F6AF7C8887C4F
:10057000627FCA3769DB1D29F86AF9503DA33A7AD0
:10058000F05FB76F3BAE0FF063F63B674F5E68AC52
:1005900024B13B84000FF3707C8D1051D0577AD476
:1005A000FB72570EB4D4CBE7E2F91E2C5C00B344C7
:1005B000AC553F11AA4700019002B8030000D24990
:1005C000737EB1C467FB020000000004595AAC00FE
:1005D000AE00AB00AD00AF00A8003A003B003C000D
:1005E0003D003E004B0000007C0000007D0000004C
:1005F0004E000100010001000100010001000100A6
:1006000001000100010001000100010001000000E3
:1006100001000000010001000100010001000100D3
:1006200001000100010001000100010001000100C2
:1006300001000000010000000100010001000100B4
:1006400001000100010001000100010001000100A2
:100650000100010001000000010000000100010094
:100660000100B005000002000200AC05000003001C
:100670000100B1050000040002009605CE06050049
:100680000100B20500000600020098050000070006
:100690000200AE05000008000100B30500000900DB
:1006A00002009A05A9060A0002009C05A9060B0093
:1006B00002009E05A9060C000200A005A9060D0077
:1006C0000200A205A9060E000200A405A9060F005B
:1006D0000200A605A90610000200A805A90611003F
:1006E0000200AA05A90612000200B40500001300CA
:1006F0000200B605000000AF00AE09025B00030176
:1007000000A0FA0904000001030101000921110100
:1007100000012240000705810308000A09040100C6
:100720000203000000092111010001222200070537
:1007300082032000010705030320000109040200D1
:10074000010300000009211101000122BC0007057E
:10075000840320000A1201000200000008646D708A
:10076000640100010203011C037600690061006C52
:10077000003A006600360034006300320062003345
:1007800000630000001003440061006D0061007010
:10079000006100640000002C0342006F006C0073D5
:1007A00000610020004B006500790062006F00616D
:1007B0000072006400200053007500700070006C2F
:1007C0000079000000040309040011241FBECFEFCC
:1007D000DAE0DEBFCDBF04B603FE27C08091AF06CE
:1007E0009091B006A091B106B091B2068730904BBF
:1007F000A740B04BD1F41092AF061092B006109201
:10080000B1061092B20614BE84B7877F84BF0FB6BC
:10081000F894A895809160008861809360001092A0
:1008200060000FBEE0E0F8E3099511E0A0E0B1E060
:10083000E0E1F9E602C005900D92AE38B107D9F7B4
:1008400026E0AEE8B1E001C01D92AF3AB207E1F791
:100850000E94F02A0C9454340C940000E8EDF0E06F
:1008600080818E7F80831092E2001092DA001092D5
:10087000E100A0EEB0E08C9181608C9380818F7755
:10088000808319BCA7EDB0E08C918E7F8C93808122
:100890008F7E808310927D0608952091E400309130
:1008A000E50095E6A9012091EC00822F817020FFE0
:1008B00006C08091E80080FF06C080E00895209186
:1008C000E80022FD1AC08091A206882389F08530B5
:1008D00089F08091EB0085FD0FC02091E4003091FC
:1008E000E50042175307F9F29150E1F684E00895CC
:1008F00082E0089583E0089581E00895EF92FF92E9
:100900000F931F93CF937C018B010E944D04C82F3E
:10091000811117C08091E80085FD0BC08091E8002F
:100920008E778093E8000E944D04882399F3C82FA6
:1009300008C0F70181917F018093F10001501109F6
:1009400049F78C2FCF911F910F91FF90EF90089551
:100950008091A40687FF13C08091E80082FF06C043
:100960008091E8008B778093E80004C08091A20614
:100970008111F2CF08958091A2068823D9F3809146
:10098000E80080FFF8CF8091E8008E77ECCF982FB9
:100990009093E900242F762F50E0891731F0709161
:1009A000EC002091ED005091F00021FD07C09F5F09
:1009B000973071F78093E90081E008953091EB0062
:1009C0003E7F3093EB003091ED003D7F3093ED00A2
:1009D0003091EB0031603093EB007093EC0020938A
:1009E000ED005093F0002091EE0027FDE0CF80E075
:1009F0000895CF92DF92EF92FF920F931F93CF93C0
:100A0000DF93C8EDD0E088818F7E8883E7EDF0E04A
:100A100080818160808384E082BF81E080937D0655
:100A200088818E7F888302EE10E0F8011082109298
:100A3000DA0081EEC82ED12CF601108288818F77E2
:100A4000888388818068888388818F7D888319BCAA
:100A50001092A2061092A3061092A1061092A00670
:100A600090EEE92EF12CF70180818B7F80838881C5
:100A70008160888342E060E080E00E94C704F60164
:100A800080818E7F8083F801808181608083808176
:100A900088608083F70180818E7F80838881806178
:100AA0008883DF91CF911F910F91FF90EF90DF909E
:100AB000CF900895FC018091AA069091AB0686170D
:100AC0009707A0F06115710529F49091E8009E77D1
:100AD0009093E80090E06115710551F4911108C000
:100AE0008091E80082FF34C080E00895BC01F2CF1D
:100AF0008091A2068823C1F18530C1F18091E80080
:100B000083FD30C08091E80082FDEACF8091E8004B
:100B100080FFE1CF8091F3002091F200382F611522
:100B2000710519F02830310558F091E02830310571
:100B300009F090E02091E8002E772093E800CBCFD9
:100B400081918093F100615071092F5F3F4FE7CF92
:100B50008091A206882341F0853041F08091E80021
:100B600083FFBECF81E0089582E0089583E0089579
:100B7000089580917F0608952FB7F89460917406C8
:100B80007091750680917606909177062FBF089533
:100B9000209123012223C9F02091780627FF15C058
:100BA000E62FE695E695E695EE31D8F4E80FF92FB5
:100BB000F11D677021E030E001C0220F6A95EAF76D
:100BC00020958281282322830895FC01329608967D
:100BD0002191621303C0DF0111971C92E817F907F6
:100BE000B9F70895209123012223C1F020917806BE
:100BF00027FF14C0E62FE695E695E695EE31F8F46A
:100C0000E80FF92FF11D677021E030E001C0220FDD
:100C10006A95EAF78281822B82830895FC013296DD
:100C20002FEF30E04191641751F02F3F19F441113B
:100C300001C0232F3F5F3630A9F72F3F09F40895F5
:100C4000820F911D27FD9A95FC01628308952091E2
:100C50007106309172062817390771F09093720669
:100C600080937106E0916F06F0917006309721F045
:100C70000084F185E02D0994089520916D0630914E
:100C80006E062817390771F090936E0680936D06F3
:100C9000E0916F06F0917006309721F00680F781A1
:100CA000E02D09940895E0916F06F0917006309759
:100CB00021F00190F081E02D099480E00895452B0A
:100CC00039F0682381E06F3F09F080E0817008957A
:100CD00081E0FCCFDC016091920580919305962F15
:100CE000891301C00895292F30E0F901EE0FFF1F8D
:100CF000E657FA4F408151814A175B07A1F487E01C
:100D00008A9FA0018B9F500D11244E5A5A4F81E0AB
:100D1000FA0184839613E6CF2F5F3F4F237033276A
:100D20002093920508952F5F3F4F922F9370D8CF55
:100D30001092EF041092EE04E2E5F5E08581811156
:100D400002C014821682379685E0EA38F807B1F7B8
:100D50000895E6E9F5E0848195812AE030E0B90163
:100D60000E949F3360931E01868180931D018285BE
:100D700080931C01848580931B0186859785B9012A
:100D80000E949F3360931A018089809319018289A0
:100D900080931801848980931701089580919605A6
:100DA000909197059093200180931F010895909151
:100DB0005904803F59F480915A0487FF0DC0109266
:100DC0005A0491110BC01092510408C0813F81F464
:100DD00080915A0418169CF3992381F080915B044A
:100DE00090915C04892B09F064C01092500408951E
:100DF000823F49F497FFF0CF1092590480915A0432
:100E00008111ECCFE0CF833F19F41916ACF3E4CF96
:100E100020915B04893F29F41216F4F610925B04CA
:100E2000DBCF8A3F19F427FFD7CFF8CF20915C049E
:100E30008B3F29F427FFD0CF10925C04CDCF8C3F9D
:100E400019F41216CCF3C8CF843F31F480915804C2
:100E50008E7F80935804C0CF853F21F48091580441
:100E60008D7FF7CF863F21F4809158048B7FF1CF9F
:100E7000873F21F480915804877FEBCF883F21F48E
:100E8000809158048F7EE5CF8D3F31F480915204DC
:100E90008E7F80935204A0CF8E3F21F48091520424
:100EA0008D7FF7CF8F3F09F097CF809152048B7FD2
:100EB000F0CF08958091520480FF0CC0609118011A
:100EC00070E075956795759567956115710549F1A0
:100ED000862F089581FF06C06091180170E0759516
:100EE0006795F3CF6091180182FD0BC0909150047B
:100EF0009923A1F06091170180911801961738F09D
:100F0000682F70E06038710500F38FE70895899FBE
:100F1000C001112470E00E94B333F4CF61E070E0AF
:100F2000D7CF81E008958091520460919E05709121
:100F30009F0580FF16C020911C01269FC001279F9E
:100F4000900D1124BC01769567957695679560386C
:100F5000710508F043C06115710509F441C0862F81
:100F6000089581FF0BC020911C01269FC001279F7F
:100F7000900D1124BC0176956795E9CF82FF09C0D9
:100F800080911C019B01829FB001839F700D1124F1
:100F9000DECF209151042223D1F290911B01809148
:100FA0001C01482F50E0291748F0CB01849FB00165
:100FB000859F700D949F700D1124C9CF289F9001BB
:100FC0001124269FA001279F500D369F500D1124FC
:100FD000692F70E0CA010E949F33B9CF8FE708954F
:100FE00081E00895803F31F40E94930781958093BA
:100FF0005A040895813F19F40E949307F8CF823F65
:1010000031F40E9493078195809359040895833F9A
:1010100019F40E949307F8CF893F29F40E945A07D8
:1010200080935B0408958A3F21F40E945A078195BA
:10103000F7CF8B3F31F40E945A07819580935C046F
:1010400008958C3F19F40E945A07F8CF843F31F479
:10105000809158048160809358040895853F21F45D
:10106000809158048260F7CF863F21F48091580424
:101070008460F1CF873F21F4809158048860EBCFE2
:10108000883F21F4809158048061E5CF8D3F31F491
:101090008091520481608093520408958E3F21F420
:1010A000809152048260F7CF8F3FB9F7809152044C
:1010B0008460F1CF80E00895F894E82FE295EF7016
:1010C000F0E031A1282F2F7081E090E001C0880F5F
:1010D0002A95EAF7982F9095932391A392A1892BB3
:1010E00082A3789408959091780692FF06C0282FE5
:1010F00028712830F9F4877F846093FF06C0282F79
:1011000028712831F1F4877E84612091790620FFCF
:1011100006C0382F38713830D9F4877F816021FFBD
:1011200006C0282F28712831D1F4877E816194FD73
:10113000877E0895282F24712430F9F68B7F8860EC
:10114000DCCF282F2471243101F78B7E8861DDCF1D
:10115000382F3171313019F78E7F8860E0CF282F1A
:101160002171213121F78E7E8861E1CFCF93DF930A
:10117000EC0182389105A9F1D8F58133910509F484
:1011800096C048F58932910509F48AC08A9709F416
:1011900095C0C11521E5D20708F0BCC0C11530E5E6
:1011A000D30708F014C1C83ED10508F09CC0C13E69
:1011B000D10560F5C83AD10508F087C0C53AD10518
:1011C00008F0FDC0C130D10509F12097F9F0C43015
:1011D000D105E0F440C08533910509F45AC0C997A0
:1011E000C1F680917806837089F0C0EED0E00EC021
:1011F000833E910599F170F4803E910501F1823EA4
:10120000910539F68091780682FD21C0CE01DF91EB
:10121000CF910895863E910561F1873E910571F168
:10122000843E910509F0B5CF8091790681FFEECF1C
:1012300080917806C7EED0E084FD0DC0E7CF8091A5
:10124000780680FD12C19091790690FFDFCFC3EE42
:10125000D0E084FFDBCFD0E0C0E0D8CF809178062B
:1012600082FD06C19091790690FDBFCF84FFCECF5D
:10127000F2CF8091780683FDDDCFC8CF80917806CC
:1012800083FDF9C09091790691FFF0CFC4EED0E0D4
:10129000BDCF8091780685FFB9CFC9E2D0E0B6CF47
:1012A0008091780685FFB2CFC5E3D0E0AFCF8091C3
:1012B000780686FFABCFCAE2D0E0A8CF809178064F
:1012C00086FFA4CFC1E3D0E0A1CFCF3BD10518F674
:1012D000C85AD0E0CC0FDD1FC15DDE4F0990D88128
:1012E000C02DD46493CFC11540E2D40758F4C11582
:1012F00081E0D80708F08ACFC03FD10508F4ABCF12
:10130000D06584CFC11590E4D90708F4A4CFDF706D
:10131000D06A7CCFC11525E5D20700F5C11534E5AB
:10132000D30708F08AC0C11543E5D40708F071C09F
:10133000C11582E5D80708F467C0CE0183709927EC
:1013400021E030E002C0220F331F8A95E2F7C695F4
:10135000C69580E2C89FE001112452C0C11599E5ED
:10136000D907A8F4C11528E5D20708F06BC0C1154C
:1013700036E5D30708F06FCF8C2F0E947308C82F73
:10138000D0E0DC2FCC27CC27DF71D0623FCFC11556
:101390004AE5D40708F45BC0CE019056811590420F
:1013A00008F059CF8D2F8F710E94730890E0982F0D
:1013B000882788279F719C012C2BE901E6CFC55A0D
:1013C000D0E0C45DDE4FC881D0E0D0641FCFCE0135
:1013D000E4E096958795EA95E1F783702C2F2695A2
:1013E0002695237040E2249F90011124382B8C2FE6
:1013F0008370C1E0D0E002C0CC0FDD1F8A95E2F718
:10140000C22BD32BDC6802CFDC2FCC27C16FD06A74
:10141000FDCECE018370992721E030E002C0220F7B
:10142000331F8A95E2F7C695C69590E2C99FE00101
:101430001124C22BD32BDA68E9CEDC2FCC27C46F62
:10144000D06AE4CEDC2FCC27C06FD06ADFCE8C2FE1
:101450008F700E94730834E0D695C7953A95E1F7EE
:10146000CF709C2FEC01D069D1CEC9E3D0E0CECEB5
:10147000C2EED0E0CBCEC6EED0E0C8CE80910D0259
:10148000882331F010920D0210920C0210920B0280
:10149000089580959091AE0698239093AE06089596
:1014A00080959091C90498239093C90408959091D0
:1014B000C904892B8093C9040895109209021092DF
:1014C000080210920702089580910602811110927D
:1014D00006020895209105029091C401291302C0CB
:1014E00080E0089530E0F90153E0EE0FFF1F5A95B8
:1014F000E1F7EB53FE4F5181561306C0508158134C
:1015000003C05281541304C02F5F3F4F2770E6CFB2
:1015100081E00895809105029091C401981301C063
:1015200008958F5F8770FACF9E3F51F1292F220FC8
:10153000E22FE90FEE0FE80F9E2F9770E695E695E4
:10154000E69583E0E89FF0011124ED54FE4F50E052
:1015500040E080E0219130E0092E02C036952795C9
:101560000A94E2F721703327042E01C0220F0A9457
:10157000EAF7822B4F5F5F4F4330510559F70895CB
:1015800080E008959E3F71F1292F220FE22FE90F8D
:10159000EE0FE80F8E2F877041E001C0440F8A954F
:1015A000EAF7E695E695E69583E0E89FF0011124D9
:1015B000ED54FE4F30E020E070E05191DF011197D3
:1015C000CB01022E02C0969587950A94E2F78170AE
:1015D00081958527842385278C932F5F3F4F233068
:1015E000310559F70895E92FE295EF70E250EE309A
:1015F00070F4F0E0EA5AFB4C0C94C733803F19F0CA
:1016000020F4883E20F481E00895843FE1F380E0F7
:101610000895883EC0F3813FD1F7F5CF93FB88272B
:1016200080F908959C013A9521153F4150F5FC0140
:10163000EE27F170BC0166277270AC01442754702C
:101640009C012227387094FF0EC080E1EF2B09F433
:1016500080E0672B09F08062452B09F08064232B22
:1016600089F08068089581E0EF2B09F480E0672B12
:1016700009F08260452B09F08460232B19F0886003
:10168000089580E00895CF92DF92EF92FF920F933A
:101690001F93CF93DF936C017B0164E670E088E7D2
:1016A0000E949E32EC0197FD12C010E000E0F601AE
:1016B000E00FF11F849164E670E00E941833EC01A2
:1016C000892B29F40F5F1F4F0E151F0581F70E940C
:1016D0009B33CE01DF91CF911F910F91FF90EF903F
:1016E000DF90CF9008958091C7049091C804911124
:1016F00003C091E089270895882369F062E070E0D3
:1017000088EF96E00E94430B892B19F08091C70463
:1017100008951092C7048091C704EBCFCF93C09176
:10172000C7048091C8048823D1F00E94BC05605A88
:1017300075418F4F9F4F6093C3047093C40480938F
:10174000C5049093C604C11108C062E070E086EF42
:1017500096E00E94430B892B29F0C091C7048C2F7F
:10176000CF91089581E08093C704F7CF80937A06E4
:1017700070937C0660937B068091A2068430F9F416
:101780008093E9008FEF9091E800815095FD06C0AD
:1017900095ED9A95F1F700008111F5CF8091E80061
:1017A00085FF0DC050E040E063E070E08AE796E01E
:1017B0000E947E048091E8008E778093E80008956F
:1017C000BC0184E00C94B60BBC0183E00C94B60B16
:1017D0009C0184E08093E9009FEF8091E8009150A4
:1017E00085FD06C085ED8A95F1F700009111F5CFD2
:1017F0008091E80085FF0CC050E040E066E070E0BA
:10180000C9010E947E048091E8008E778093E800F1
:101810000895CF93DF93EC01809123018823B1F1E8
:101820008091780687FF32C060E284E08093E9000F
:101830008FEF9091E800815095FD06C095ED9A9547
:10184000F1F700008111F5CF8091E80085FF1BC002
:101850008091230170E050E040E0811104C050E02D
:1018600040E068E070E0CE010E947E048091E800D4
:101870008E778093E80080E2FE01A0E8B6E0019058
:101880000D928A95E1F7DF91CF91089568E081E0AC
:10189000CDCF81E08093E00080E28093D800109269
:1018A000C9008FE19EE40197F1F700C0000087E0D6
:1018B00090EBDC018093AF069093B006A093B10645
:1018C000B093B20688E19CE00FB6F894A895809397
:1018D00060000FBE90936000FFCF019708F4089559
:1018E000EFE9FFE03197F1F700C00000F6CF0F936A
:1018F0001F93CF93DF9306E915E0C7ECD0E0CE014C
:101900000E940A34F80181938F012196C93ED105C6
:10191000B1F7C4E6D6E0FE0185919491009711F0ED
:10192000FC0109952896F6E0CC3FDF07A1F7DF918F
:10193000CF911F910F9108950F931F93CF93DF9332
:10194000843000F561111EC024E0829F80011124C3
:1019500050E0440F551F040F151F09541F4FC801B5
:101960000E940A34C82FD0E0DC2FCC27C801019692
:101970000E940A349E01282BC901DF91CF911F914B
:101980000F91089590E080E0F8CF0F931F93CF93CD
:10199000DF93843030F5633020F5463010F5C42FE6
:1019A000D0E0CC0FDD1F2CE0629FC00DD11D1124B3
:1019B00034E2839FC00DD11D1124CE0187960E9471
:1019C0000A34082F10E0102F0027CE0188960E94BD
:1019D0000A349801282BC901DF91CF911F910F91F3
:1019E000089590E080E0F8CF462F2091C104309117
:1019F000C204232B91F47E3F39F46E3F71F4809141
:101A0000BF049091C0040895843038F4733028F4F2
:101A1000663018F4672F0C94C50C90E080E00895B0
:101A2000CF92DF92FF920F931F93CF93DF936C01BE
:101A30000091AD068091AC06082BC7E0D0E010E025
:101A4000FC2EC8010C2E02C0959587950A94E2F7EA
:101A500080FD0CC02197A0F7F12C8F2DDF91CF9145
:101A60001F910F91FF90DF90CF900895B6018C2FBA
:101A70000E94F40C0E94B608019761F3EECFCF9359
:101A8000DF93EC010E94100DBE010E94F40CDF9167
:101A9000CF910C94B608FC0186819781009721F0C4
:101AA0000E94B6080C94F30A808191810E943F0D38
:101AB000F9CF1F93CF93DF9300D000D00F92CDB713
:101AC000DEB749835A8389819A816623B9F022233C
:101AD000A9F00E94100D182F682F89819A810E9409
:101AE000C20A69817A81812F0F900F900F900F9019
:101AF0000F90DF91CF911F910C94F40C0E94940AE7
:101B0000182FEFCFFC01262F86819781009739F49B
:101B1000408151816281738184810C94590D0895B3
:101B200083E290E00E940A348B3B89F484E290E0E7
:101B30000E940A34863459F485E290E00E940A3407
:101B400091E08C3609F090E0892F8170089580E053
:101B5000FCCFCF9384E090E00E940A34C82F82E249
:101B600090E00E940A34982F8C2FCF9108950F9304
:101B70001F93CF93DF9306E915E0C7ECD0E0CE01C9
:101B80000E940A34F80161918F01681719F0CE01A3
:101B90000E9418342196C93ED10589F7DF91CF9173
:101BA0001F910F910895E6E9F5E0128E138E8FEAEA
:101BB00090E09183808385E0848F88E893E193832C
:101BC00082834CE251E05583448322E330E0378343
:101BD000268385E090E0918780878AE090E0938774
:101BE000828764E170E0758764875787468744E69B
:101BF00050E0518B408B48E050E0538B428B48E2E1
:101C000050E0558B448B378B268B28EC30E0318F9E
:101C1000208F158E978F868F80E590E091A380A30B
:101C20000E94B70D0C94770CCF93DF93C9E8D1E0F5
:101C300060E0CE010E9418342196C11584E0D807D7
:101C4000B9F7DF91CF9108950F931F93CF93DF934F
:101C50008901843028F5611123C0423008F521152F
:101C60003C4531F42091150130911601232BC1F030
:101C700094E0899FE001112450E0440F551FC40FE8
:101C8000D51FC954DF4F612FCE010E941834602F39
:101C9000CE010196DF91CF911F910F910C941834D2
:101CA000DF91CF911F910F9108950F931F93CF93C1
:101CB000DF938901843048F5633038F5463028F5E4
:101CC00021153C4531F42091150130911601232B4B
:101CD000E1F0C42FD0E0CC0FDD1F9CE0699FC00D68
:101CE000D11D112494E2899FC00DD11D1124612FB3
:101CF000CE0187960E941834602FCE018896DF911E
:101D0000CF911F910F910C941834DF91CF911F91B7
:101D10000F910895CF93C82F6FEF81116BEB83E282
:101D200090E00E9418346FEFC11166E484E290E005
:101D30000E9418346FEFC1116CE685E290E0CF91FC
:101D40000C9418347F928F929F92AF92BF92CF9251
:101D5000DF92EF92FF920F931F93CF93DF93CDB754
:101D6000DEB764970FB6F894DEBF0FBECDBFA0906C
:101D70001501B090160181E090E0909316018093D8
:101D800015018EECC82E85E0D82E10E0760100E01B
:101D900015C0F40125913491472D602F812F0E94A9
:101DA000550E82E0880E911C7394E6E07E12F1CF0E
:101DB000FCE0EF0EF11C0F5F033019F04701712CAE
:101DC000E8CF21E030E040E060E0812F0E94240E67
:101DD00021E030E041E060E0812F0E94240E1F5F8F
:101DE00084E2C80ED11C143089F60E94D30D1A82E9
:101DF00019821C821B821E821D8218861F8288EC1B
:101E000090E09A87898709EE10E04AE050E0B80137
:101E1000CE0101960E943C34065F1F4F0933E1E07A
:101E20001E0799F77E01FBE0EF0EF11C8AE0F70137
:101E300011928A95E9F74AE050E0B801C7010E9483
:101E40003C34065F1F4F0938F1E01F07A1F7B0923D
:101E50001601A092150164960FB6F894DEBF0FBE6E
:101E6000CDBFDF91CF911F910F91FF90EF90DF9049
:101E7000CF90BF90AF909F908F907F90089580E01B
:101E80000E948A0E60E086E290E00E9418340E9470
:101E9000A20E0E94140E81E00C948A0E9B018830E1
:101EA00070F49AE0899FB001112467517F4F4AE096
:101EB00050E0C9010E94FA3390E080E008958FEF6E
:101EC0009FEF08958F929F92AF92BF92CF92DF9231
:101ED000EF92FF920F931F93CF93DF93CDB7DEB7AF
:101EE0002A970FB6F894DEBF0FBECDBF0DEB15E0FD
:101EF000F12CE12C83E2C82E8AE2D82E9DE4A92E93
:101F00009AE2B92E2BE3822E29E2922EF801D18299
:101F1000C082B382A28295828482F58AE48ABE015D
:101F20006F5F7F4F8E2D0E944E0F892B29F489857C
:101F30009A85F801938B828BFFEFEF1AFF0A0A5EF6
:101F40001F4F88E0E816F10409F72A960FB6F894B7
:101F5000DEBF0FBECDBFDF91CF911F910F91FF90DC
:101F6000EF90DF90CF90BF90AF909F908F900895AB
:101F7000CF92DF92EF92FF920F931F93CF93DF9355
:101F8000CDB7DEB72A970FB6F894DEBF0FBECDBF30
:101F9000EFE6F4E080E5DF011D928A95E9F7E2E5DE
:101FA000F5E088E3DF011D928A95E9F78FE6C82EF8
:101FB00084E0D82E7F0109E311E0F701D182C082CD
:101FC0004AE050E0B801CE0101960E94FA3388E061
:101FD000FE013196D60101900D928A95E1F789852F
:101FE0009A85D70113969C938E931297BAE0CB0EE5
:101FF000D11CE7E0EE0EF11C065F1F4F0938F1E03F
:102000001F07D9F62A960FB6F894DEBF0FBECDBFD4
:10201000DF91CF911F910F91FF90EF90DF90CF90C4
:1020200008956AEE7EEF90E080E00E94363460E032
:1020300082E090E00E94183460E083E090E00E942B
:1020400018341092AC0660E084E090E00E941834EE
:1020500060E082E290E00E94183460E085E090E069
:102060000E94183460E086E090E00E9418346FEF20
:1020700087E090E00E94183440E050E0BA0188E028
:1020800090E00E942A3460E08DE090E00E941834D5
:1020900040E050E0BA0188E190E00E942A3460E01C
:1020A00087E190E00E94183440E050E0BA018CE1F2
:1020B00090E00E942A3470E060E080E290E00E94AC
:1020C000363440E050E0BA0188E190E00E942A34C2
:1020D00080E00E948A0E0E943F0F40E050E0BA016B
:1020E0008FE090E00E942A3440E050E0BA0183E1A2
:1020F00090E00C942A341F920F920FB60F92112485
:102100002F933F934F935F936F937F938F939F93FF
:10211000AF93BF93EF93FF938091E10082FF09C0DB
:102120008091E20082FF05C08091E1008B7F809367
:10213000E1008091DA0080FF24C08091D80080FF08
:1021400020C08091DA008E7F8093DA008091D900E0
:1021500080FF9DC080E189BD82E189BD09B400FE98
:10216000FDCF81E08093A20680917D06811109C098
:102170000E942E040E94F9048091E2008460809302
:10218000E2008091E10080FF17C08091E20080FFB3
:1021900013C08091E2008E7F8093E2008091E20084
:1021A00080618093E2008091D80080628093D800A3
:1021B00019BC85E08093A2068091E10084FF2BC0CA
:1021C0008091E20084FF27C080E189BD82E189BD62
:1021D00089B5982F917080FFFBCF8091D8008F7DBB
:1021E0008093D8008091E1008F7E8093E100809100
:1021F000E2008F7E8093E2008091E2008160809314
:10220000E2008091A306882309F447C084E080930C
:10221000A2068091A2068091E10083FF27C08091F1
:10222000E20083FF23C08091E100877F8093E1007B
:1022300082E08093A2061092A3068091E1008E7F37
:102240008093E1008091E2008E7F8093E200809194
:10225000E20080618093E20042E060E080E00E9462
:10226000C7048091F00088608093F000FF91EF91A7
:10227000BF91AF919F918F917F916F915F914F919E
:102280003F912F910F900FBE0F901F90189519BC82
:102290001092A20610927D0674CF8091E30087FD14
:1022A00093E09093A206B5CF78941F921FB61F9229
:1022B00011248F939F93AF93BF9380917406909155
:1022C0007506A0917606B09177060196A11DB11D05
:1022D0008093740690937506A0937606B093770664
:1022E000BF91AF919F918F911F901FBE1F90189526
:1022F0009C014FB7F8948091740690917506A09157
:102300007606B09177064FBF821B930B08952FB7C7
:10231000F8948091740690917506A0917606B0911C
:1023200077062FBF08950E9487119C019091590450
:1023300080915A04982B21F0309356042093550431
:1023400090915B0480915C04982B21F030935404AD
:1023500020935304E0916F06F0917006309749F096
:1023600082E0809357040480F581E02D87E594E0B6
:1023700009940895CF93C82F8091790682FD0CC0EF
:1023800080910D028C1741F00E94871190930C02EE
:1023900080930B02C0930D02CF9108958091980510
:1023A00090919905892B89F00E94871120910B0249
:1023B00030910C02AC01421B530B81E02091980537
:1023C000309199054217530708F480E08170089511
:1023D0008091C9049091AE06892B90910A02892BB5
:1023E0008093900180910D02882319F180919805C6
:1023F00090919905892B29F00E94CE1181110E949C
:102400003E0A8091900190910D02892B809390015A
:1024100080912301882341F18091780687FF24C0B1
:102420008EE1E2E9F1E090E0815000F591110E9427
:102430003E0AE0916F06F09170063097E1F08091CE
:102440002301882359F08091780687FF07C0809187
:1024500090018093910186E0809390010280F38146
:10246000E02D80E991E0099486E0DBCF21912223E1
:10247000D9F29F5FD9CF0895EF92FF920F931F93E8
:10248000CF93DF93EC018A85811134C0EB80FC800F
:1024900087E5F81A26E12E9DC0012F9D900D11248D
:1024A000DC01A354BA4F1496ED91FC911597309727
:1024B00031F054966D917C918D539A4F099586E138
:1024C0008E9D80018F9D100D112403541A4FF80129
:1024D00087810E94500AF80180850E94490A0E9463
:1024E000E811188219861B861E821D821092BC0577
:1024F0001092BB05DF91CF911F910F91FF90EF904C
:102500000895CF93DF93EC018989811118C081E090
:10251000898B8F810E94570A8091AE069885892BFE
:102520008093AE060E94E811EA81FB81309739F072
:102530006C897D89CE010696DF91CF910994DF9158
:10254000CF91089580912101877F8093210182E0BE
:102550000E94490A8091210184FF06C08F7E8093EA
:10256000210182E00E94570A8091210185FF06C067
:102570008F7D8093210180E20E94570A0C94E8111C
:1025800090E080E00E943D0690E080E00E942706F7
:102590001092AE0610920A020E94E81186E0E7E56A
:1025A000F4E0DF011D928A95E9F710925104109230
:1025B0005004109252040C9493118093AD060C9425
:1025C000C0128091AD06982F9670963019F48860ED
:1025D0000C94DD12877FFCCF21E030E001C0220F98
:1025E0008A95EAF720958091AD0682230C94DD123E
:1025F000909109028095892380930902282F2770E2
:1026000091F4282F082E000C330B9217130659F063
:102610009091790692FD07C08595859585950E94D4
:10262000EC120C945D0A0895CF93C0917906C2FB19
:10263000992790F9981799F080FBC2F9C093790611
:102640006091780684E090E00E9418346C2F82E25A
:1026500090E00E94183482E0CF910C94F812CF9150
:10266000089521E030E001C0220F8A95EAF78091B9
:10267000AD06822B0C94DD129091790692FD10C06C
:1026800098E0899F90011124622B609309020E94B7
:1026900031130E94871190930802809307020895D6
:1026A0000C9431138093AC060C94C0121092C904A0
:1026B00080912301E2E9F1E0882359F080917806C6
:1026C00087FF07C08EE1DF011D928A95E9F70C9420
:1026D000C01286E0F8CF1F93CF93DF93CDB7DEB75C
:1026E000AA970FB6F894DEBF0FBECDBF84EA96E07E
:1026F0002091F100DC012D93CD01B6E08C3A9B07CF
:10270000B9F78091A506833009F472C0B8F481301E
:1027100009F449C0823009F4B3C08091E80083FF16
:1027200096C28091A4069091A5069A3008F08FC2B7
:10273000E92FF0E0EC59FB4C0C94C7338A3009F4D4
:102740008EC08B3009F471C0893039F78091A406AE
:10275000813219F78091A8069091A906009711F08F
:102760000297D9F68091E800877F8093E8008091F6
:10277000E80082FF38C09091F3008091F200029748
:1027800031F48091F100813011F0863021F4809194
:10279000F10080937F068091E8008B778093E800BA
:1027A0000E94A804BACF8091A406813A09F0B5CF5F
:1027B0008091E800877F8093E8008091A80690913F
:1027C000A906892B61F460E280E896E070E00E943F
:1027D0005A058091E8008B778093E8009ECF60E0F7
:1027E00090E080E0F3CF8091A2068111C0CF95CF19
:1027F0008091A406813A09F090CF8091A80690912B
:10280000A906892B09F089CF8091E800877F809302
:10281000E8008091E80080FFFCCF80912301809345
:10282000F1008091E8008E77B9CF8091A4068132C3
:1028300009F073CF8091A8069091A906892B09F021
:102840006CCF8091E800877F8093E8000E94A80405
:102850008091A606809323010E9456135ECF80913B
:10286000A406813209F059CF8091E800877F8093D8
:10287000E8000E94A8048091A70680937E064DCFB1
:102880008091A406813A09F048CF8091E800877FC3
:102890008093E8008091E80080FFFCCF80917E0665
:1028A000BECF803899F0823809F0D1C18091A80656
:1028B0008F70873008F0CBC18093E9008091EB00E6
:1028C00085FB882780F91092E90006C08091A00658
:1028D0009091A106911182609091E800977F90936A
:1028E000E8008093F1001092F1008091E8008E776B
:1028F000AAC1882309F498C1823009F0A8C1809147
:10290000A60681119BC18091A8068F702FEF280F1A
:10291000263008F09CC18093E9002091EB0020FF55
:102920008DC1933031F48091EB0080628093EB0095
:1029300085C19091EB0090619093EB0021E030E035
:1029400001C0220F8A95EAF72093EA001092EA006C
:102950008091EB008860EACF811179C11091A606C1
:102960001F778091E3008078812B8093E300809132
:10297000E800877F8093E8000E94A8048091E80027
:1029800080FFFCCF8091E30080688093E30082E0C9
:10299000111183E08093A2065AC18058823008F05A
:1029A00056C12091A6063091A7062C3DE3E03E07D4
:1029B000A1F583E08A838AE289834FB7F894DE0128
:1029C000139620E03EE051E2E32FF0E050935700F1
:1029D000E49120FF03C0E295EF703F5FEF708E2F10
:1029E00090E0EA30C0F0C7968D939D932F5F24311D
:1029F00059F74FBF8091E800877F8093E8006AE233
:102A000070E0CE0101960E945A058091E8008B7714
:102A10008093E8001CC1C096E7CF8091A8069091F2
:102A2000A906432F55274330510509F44AC078F5CC
:102A30004130510509F485C08BE590E0EAEFF6E0FE
:102A40004230510509F003C12091E800277F20930F
:102A5000E8002091AA063091AB068217930708F48C
:102A60009C0140E02115310509F070C041116EC094
:102A70008091E80082FDC9CF8091A206882329F2C7
:102A8000853019F28091E80083FFF2CFBECF41324A
:102A9000510509F447C04232510509F0D8C08330CE
:102AA000910508F0D4C0FC01EE0FFF1FEF57FE4F59
:102AB0000190F081E02D82589E4FDC018C9190E0D6
:102AC0001DC0332721303105E9F02115310579F09A
:102AD00022303105F9F02330310509F0B8C0E7E6BE
:102AE000F7E0E4918E2F90E0E7E6F7E007C0E5EC31
:102AF000F7E0E4918E2F90E0E5ECF7E0009709F421
:102B0000A6C0A2CFE7E9F7E0E4918E2F90E0E7E9D5
:102B1000F7E0F4CFE5E8F7E0E4918E2F90E0E5E808
:102B2000F7E0ECCF8330910508F091C0880F991F32
:102B3000FC01E957FE4F0190F081E02D89E090E023
:102B400083CF82E190E0E5E5F7E07ECF8091A206B9
:102B5000882309F45ACF853009F457CF8091E800D3
:102B600083FD53CF8091E80082FD82CF8091E80001
:102B700080FF78CF9091F3008091F200211531050C
:102B800019F08830910550F041E0089709F040E0D5
:102B90008091E8008E778093E80064CF4491409361
:102BA000F1003196215031090196E8CF803809F0C3
:102BB0004EC08091E800877F8093E8008091A30653
:102BC0008093F10092CE811142C01091A60612307E
:102BD000F0F58091E800877F8093E8001093A306CA
:102BE0000E94A804112311F084E005C08091E30045
:102BF00087FDFACF81E08093A20642E061EC81E09C
:102C00000E94C70442E261EC84E00E94C70442E2F1
:102C100061EC82E00E94C70442E260EC83E00E9423
:102C2000C7048091A20613C08091A606813079F472
:102C300081E0933009F080E08093A1061092E900D2
:102C40008091E800877F8093E8000E94A80480912B
:102C5000E80083FF0AC08091E800877F8093E80046
:102C60008091EB0080628093EB00AA960FB6F894F7
:102C7000DEBF0FBECDBFDF91CF911F9108951F9290
:102C80000F920FB60F9211242F933F934F935F93A0
:102C90006F937F938F939F93AF93BF93CF93DF9364
:102CA000EF93FF93D091E900DF708091EC00C82F83
:102CB000C17080FDC0E81092E9008091F000877F2C
:102CC0008093F00078940E946B131092E900809139
:102CD000F00088608093F000CD2BCF70C093E900A6
:102CE000FF91EF91DF91CF91BF91AF919F918F9124
:102CF0007F916F915F914F913F912F910F900FBEF8
:102D00000F901F901895882321F00E94490A0C9477
:102D1000E8110895882339F09091AE06982B90938E
:102D2000AE060C94E8110895882321F00E94500A01
:102D30000C94E8110895882321F00E94570A0C94FE
:102D4000E8110895882379F19CEF980F913A38F4AF
:102D5000682F80E991E00E94C8050C94E81190E288
:102D6000980F983050F4877091E001C0990F8A95C0
:102D7000EAF7892F0E94500AF0CF9BE5980F933015
:102D800020F490E080E00C943D0698E5980F973190
:102D900020F490E080E00C942706803F20F00E9411
:102DA000D7060C9493110895CF93DF93EC010E9402
:102DB000A216CE010E94120B9E01205E310928301E
:102DC000310510F0CD2B21F4DF91CF910C949416A6
:102DD000DF91CF910C948316CF93C82F882309F4E9
:102DE0006BC08CEF8C0F813AC0F580912301882352
:102DF00011F18091780687FF1EC0EC2FE695E695CD
:102E0000E695F0E0E057FE4F828190E04C2F47704E
:102E100021E030E002C0220F331F4A95E2F78223FF
:102E20009323892B91F06C2F80E991E00E94C805D3
:102E30000E94E8110AC0E2E9F1E088E991E02191FD
:102E4000C21789F38E179F07D1F76C2F80E991E0A5
:102E50000E94F205CF910C94E81180E28C0F88302B
:102E600048F4C77081E001C0880FCA95EAF70E9454
:102E7000570AF0CFEBE5EC0FE33040F4F0E0E45D0F
:102E8000FE4F808190E0CF910C943D06E8E5EC0F79
:102E9000E73150F4F0E0EE0FFF1FE15DFE4F80815F
:102EA0009181CF910C942706C03F30F08C2F0E9467
:102EB000F207CF910C949311CF9108951F93CF9364
:102EC000DF93182FC091B605D091B705893321F053
:102ED000C091B405D091B505812F0E94EC162097C2
:102EE00031F4812FDF91CF911F910C94A2168FE9BD
:102EF0009FE00197F1F700C000002197F0CF0F93FA
:102F00001F93CF93DF93C42FD22FFC01828188239C
:102F1000A1F04093BA050E9487119093B905809360
:102F2000B805C77081E001C0880FCA95EAF7DF9144
:102F3000CF911F910F910C949B161091BA05141309
:102F400039C08091B8059091B9050E9478112091FF
:102F5000AE053091AF058217930760F5C0E2CD0F43
:102F60001D17B9F080E2810F883040F4177081E0BE
:102F700001C0880F1A95EAF70E949416C83048F4E9
:102F800081E09D2F977001C0880F9A95EAF70E9403
:102F90009B16802F0E945E17C83098F4D77081E08E
:102FA00001C0880FDA95EAF7DF91CF911F910F9159
:102FB0000C949416C77081E001C0880FCA95EAF797
:102FC000F3CFDF91CF911F910F910895AF92BF92F0
:102FD000CF92DF92EF92FF920F931F93CF93DF93E5
:102FE000EC018AE0A82E2881222309F48CC021302C
:102FF000C9F599818A81913021F422960E945E1749
:1030000005C0923029F422960E94EC162196EBCF4F
:10301000933021F422960E94A216F8CF943011F03A
:103020002196F4CF229630E020E0AE014F5F5F4F53
:103030008053990B8A30910550F02150310930F3BB
:103040008FE99FE00197F1F700C00000F6CFA29E44
:10305000B001A39E700D11249C01260F371F89819A
:10306000EA01E3CFE22FF0E0E650FE4FB490822F6A
:1030700086958695869590E0FC01E651FE4FE4909A
:103080002770F12C022E02C0F594E7940A94E2F71F
:1030900031E0E322FF24FC01E652FE4FC490D12C24
:1030A000022E02C0D594C7940A94E2F731E0C322FD
:1030B000DD24FC01E653FE4F049110E002C015959B
:1030C00007952A95E2F701701127E114F10419F030
:1030D00081EE0E94EC16C114D10419F086EE0E9414
:1030E000EC168B2D0E945E17CD2819F086EE0E94FB
:1030F000A216EF2819F081EE0E94A216012B09F406
:1031000085CF8CE27BCFDF91CF911F910F91FF9004
:10311000EF90DF90CF90BF90AF900895CF93DF9363
:10312000EC010E94120B9E01205E3109283031050E
:1031300010F0209739F40E949B168C2FDF91CF91CD
:103140000C94EC160E948A16F8CF662329F0209181
:10315000AE0622602093AE069C013056211540E257
:10316000340720F0305E2115304108F499270C9483
:103170008E18DF92EF92FF920F931F93CF93DF93FE
:103180007C018B01D42E8091210182FF8CC0C091E3
:10319000EC04D091ED04CE15DF0521F0E114F1042B
:1031A00009F081C0809121018B7F8093210181FDF5
:1031B00073C08091EA049091EB04A801481B590B5D
:1031C00081E020911F01309120014217530708F43C
:1031D00080E08170F82E80912101F0FA81F98093CE
:1031E0002101FE0183E0F695E7958A95E1F7EE71FE
:1031F000FF27E653FB4F20813181AE014F705527E9
:1032000081E090E002C0880F991F4A95E2F7FF2005
:1032100009F444C0822B932B918380838091C9044D
:1032200081FF08C08091210180618093210182E0AB
:103230000E94500A8091C90485FF08C08091210135
:1032400080628093210180E20E94500A6F2DCE019E
:103250000E94A518DD2031F08091B10585FF02C0E4
:1032600086FF3BC08091B4059091B5050E946D0C1E
:103270008091EC049091ED049C013056211540E2C0
:10328000340720F0305E2115304108F499270E9460
:10329000D4160E94A2121DC081E09BCF809590950C
:1032A00082239323B9CFC70199279701305621155F
:1032B00040E2340728F0305E2115304108F0C701A4
:1032C0000E94D4168091EC049091ED048E159F0518
:1032D00001F31093EB040093EA04DF91CF911F9167
:1032E0000F91FF90EF90DF9008958F929F92AF9291
:1032F000BF92CF92DF92EF92FF920F931F93CF93E3
:10330000DF9300D000D0CDB7DEB77C01DC0113968F
:103310004D915C91149711966C9111978C910E942C
:103320005F06811179C061E0C7010E94820D8C01A6
:10333000F7018281811111C0D70112968C91811100
:1033400049C00031FFE51F0709F4EEC001312FE548
:10335000120709F007C782E0E8C080910001909150
:103360000101019649F36DEBC62E65E0D62EB12C16
:10337000A12C9924939480910001909101018A15C8
:103380009B05D4F2F60186818823E9F08185928538
:103390000817190739F48091BB059091BC050817EF
:1033A000190789F0D6011F969C921F971C961C93B3
:1033B0000E931B97C6010E948112C60106960E94B9
:1033C0003C121092AE06BFEFAB1ABB0AE6E1CE0E7E
:1033D000D11CD1CF980122513F452031310508F051
:1033E000B7C68FEF93E00E940A345EEED52ED00E62
:1033F00009E811E0882369F180910902877061F082
:10340000D70112968C91882339F08091790682FD3C
:1034100003C082E00E94F8120F900F900F900F905F
:10342000DF91CF911F910F91FF90EF90DF90CF90A0
:10343000BF90AF909F908F9008950115F4E01F0703
:10344000D9F2C8010E940A34811101C0DA940F5FD9
:103450001F4FD110F2CF19821A821B821C82CC24FA
:10346000CA9448012FEF821A920AC8010E940A34B6
:1034700089831A82882309F4BFCF813009F048C0BC
:10348000580132E0A30EB11CC4010E940A34982EE8
:103490008A83882309F4B0CFC5010E940A34D82E4C
:1034A0008FEF890D833068F4580143E0A40EB11CFE
:1034B000DB82DD2021F0CE0101960E94E617850116
:1034C000D0CF54E09512FBCF580184E0A80EB11C78
:1034D000C80103960E940A34DD2009F48DCF8823A9
:1034E00009F48ACF8150990BC89E9001C99E300D76
:1034F0001124AD2DA150BB0BCD01820F931F01975D
:10350000F0F2EFE9FFE03197F1F700C00000F7CFEC
:10351000CE0101960E94E6175401D1CF81E00E94AE
:1035200031130E94E11268CF81E00E94EC12F9CFC2
:1035300082E0F5CF4FEFC416D10411F008F01EC69B
:1035400065E674E08C2D0E944E0F892B29F586E1EB
:103550008C9DF0018D9DF00D1124E354FA4F86816E
:10356000813009F062C08091650490916604892BD6
:1035700099F08091670490916804892B69F080919B
:10358000690490916A0420916B0430916C04822B41
:10359000932B892B09F453C0809100019091010174
:1035A0008C159D0524F4D0920101C0920001F70111
:1035B000828196E19C9D50019D9DB00C1124950146
:1035C00023543A4F6901D90150968C9350979281B8
:1035D00016968C911697992309F43FC01A961C935E
:1035E0000E9319978F5F16968C930E948711F601A0
:1035F0009687858780910D0287838091AE06909192
:10360000C904892B80870190F081E02D309741F02B
:10361000D60154966D917C91C5018D539A4F0995B1
:103620001093BC050093BB05A9C5823009F0B4CF47
:103630008091690490916A04892B09F4ADCF26E149
:103640002C9DC0012D9D900D112483549A4FDC01B7
:1036500050961C920E9481129FCF882309F48EC538
:10366000F9018189882309F489C5C5018D539A4FD1
:103670000E943C1283C580912101816080932101C9
:10368000ABC5809121018E7F809321010E94A212FF
:10369000A3C5809121018F7E013E110531F0053EC9
:1036A0001105C9F4809121018F7D809321018091C2
:1036B000210180FFA0C5D70112968C910832110517
:1036C00028F50E31110508F074C00430110580F59D
:1036D00081118DC590C5C8019056811540E29407AF
:1036E00020F0905E8115904110F78091210182FFBA
:1036F00082C58091B30581FD7EC521E132E040E0C5
:10370000B60190E080E00E94B91875C50933110533
:1037100058F40D32110518F40B321105C9F69091C9
:10372000B10592FDD5CF08C004361105C1F3D0CF45
:103730009091B10594FDCCCF882309F4A1C090915C
:10374000C90480910D02282F292B322F3D7FB1F122
:103750001092ED041092EC043091B10531FD2EC0B1
:10376000F80143E0F695E7954A95E1F7EE71FF27FA
:10377000E653FB4F98012F70332781E090E002C0A1
:10378000880F991F2A95E2F78095909520813181C5
:10379000822393239183808360E0C8010E94A5184F
:1037A00080910D028D7F0E94BA1182E00E94F81272
:1037B00023CE9091B10593FD8BCFBECF38E0F701BA
:1037C000A1E1B2E001900D923A95E1F71092130257
:1037D0001092150210921402A090EC04B090ED0427
:1037E0000A151B05B1F53091B10535FF32C0409186
:1037F000210141FB992490F841FF02C036FF29C006
:103800004091EA045091EB04B601641B750B4091A2
:10381000AE055091AF0564177507D8F491FF08C045
:103820008091210180618093210182E00E94500AF1
:103830008091C90485FF08C0809121018062809336
:10384000210180E20E94500A692DC5010E94A5183D
:10385000D3CD9091210121FB91F9909321018D7F8E
:103860000E94BA111093ED040093EC04D092EB0483
:10387000C092EA048091210184608093210195CF58
:10388000970140E0B601C8010E94B918B5CD053FC7
:103890004CE5140709F467C008F45FC0063F8CE5E7
:1038A000180709F466C0D70112963C91332309F436
:1038B000C1C41092BA050330BDE51B0708F065C00E
:1038C0000A3FECE51E0730F4C80182509C4544973E
:1038D00008F060C00E94A90D909379068093780645
:1038E00000312CE5120709F461C108F0DDC0083091
:1038F0004CE5140709F448C108F0AFC004308CE56A
:10390000180709F433C108F095C00230ACE51A0776
:1039100009F426C180917806826003301C4509F4C1
:1039200022C1609178061091790684E090E00E94AF
:103930001834612F82E290E00E9418340E945613DE
:103940005BCD07E225EE45EE68ED7CE56FC406E24F
:1039500021EE40EE63EF7CE569C407E225EE44EE1C
:1039600064EF7CE563C406E221EE42EE65EF7CE5A0
:103970005DC407E225EE46EE66EF7CE557C408E23B
:1039800021E045EE69ED7CE551C40136FDE51F07F8
:1039900009F4A0CF06315CE5150709F44FC40A35D8
:1039A0004DE5140709F453C108F02FC101158CE54A
:1039B000180709F43CC10E3D1C4509F445C1F70147
:1039C00086819781009709F446C10E94B608182F96
:1039D000092FF701D280C580C2943FE0C3228091B5
:1039E00009028770C1F0AD2CDD20B1F0892F807FF6
:1039F000803421F080E2810F883068F08091790670
:103A000082FD09C082E00E94F8128091090287704D
:103A1000AA24A3948111A12C902E92942FE092229B
:103A2000FBE0F91508F4A4C1E92DF0E0E259FB4CE4
:103A30000C94C7338091780680610630ECE51E0750
:103A400009F491C080917806886007301C4508F41D
:103A50008AC080917806806286C0809178068D7FCA
:103A60000C302CE5120709F47EC070F480917806C2
:103A70008C600A304CE5140709F475C008F488C05E
:103A8000809178068E7F6FC00E308CE5180709F4A0
:103A900085C0809178068B7F0F301C4508F463C089
:103AA000809178068F7E5FC00C3FACE51A0709F461
:103AB00079C068F50431ECE51E0709F48BC080F489
:103AC00002312CE5120709F475C0809178068F7BCE
:103AD00003311C4508F447C080917806837F43C0BA
:103AE0000A3F4CE5140709F445C008F049C0053108
:103AF0001C4509F016CF8091780682FB992790F932
:103B000021E0922790FB82F990FB83F92CC00115EC
:103B10009DE5190709F454C088F480917906836003
:103B20000E3FBCE51B0749F1809179068D7F0F3F61
:103B30001C4518F1809179068C7F1FC00230FDE58D
:103B40001F0709F456C008F44EC001361D4509F0A0
:103B5000E8CE90917806892F8F7E94FF806103C014
:103B600080917806816080937806DBCE809178061C
:103B70008460F9CF80917906816080937906D1CEF7
:103B8000809179068260F9CF809178068064EBCFCE
:103B90000E945613809178068068E5CF8091780660
:103BA000877FE1CF809179068E7FE7CF809178067D
:103BB0008F7DD9CF0E945613809178068F77D3CF0F
:103BC00080917906982F909591708E7F892B90FB2C
:103BD00081F9D3CF0E94561390917806892F97FBD5
:103BE00087F98058C0CF61E08EE090E00E941834E1
:103BF00098CE60E0F9CF8091B00169E2811165E370
:103C000080E991E00E94C80546C30B35ADE51A076F
:103C100001F10C351D4509F0D2CE8091790682FB69
:103C2000882780F991E089270E941413C8CE0E944A
:103C30005613EFEFF4E32CE0E150F0402040E1F7C1
:103C400000C000000E94490C0E941110D5CB81E0F9
:103C5000EBCF80E0E9CF828100811181882369F078
:103C6000C8010E94100DD82E682FC8010E94C20AF8
:103C7000B8018D2D0E94F40CA8CEC8010E94940AB0
:103C8000D82EF6CF202F2F70B22E802F807F19F0E4
:103C9000B29490EFB922DD20A9F0BB2059F080E268
:103CA000810F883010F0111107C08B2D0E94570A28
:103CB0000E94E811812F5AC08091AE06B82AB092B6
:103CC000AE06F6CF812F0E94A216BB2009F450C089
:103CD00080E2810F883010F0111104C08B2D0E94FA
:103CE000500A03C08B2D0E94490A0E94E81140C06F
:103CF000302F3F70B32E802F807F803219F0B29426
:103D000080EFB822112321F1113009F4A4C0DD2085
:103D100009F4ADC0CC2009F47DC020E0D7014C915E
:103D200011965C91119712966C91129713967C9153
:103D3000139714968C910E94590D8091B30581FDC3
:103D4000B9CFF701858180FFB5CF8F70858362C0C1
:103D50008091790682FF40C0DD20C1F1BB2029F0AF
:103D60008B2D0E94570A0E94E81180E00E94EC16F9
:103D7000A92DA850BB0B149710F40E945306812F55
:103D8000902F0E94F30A8111C4C11092B2011092C7
:103D9000B101AA20B1F08091090280FD12C0D701C3
:103DA00012961C928595859585950E943113C701C1
:103DB0000E947519809109028595859585950E94C7
:103DC000EC1260E0C7010E94820D26CB80E00E94C9
:103DD000A216BB2069F282CFDD2001F1C11004C020
:103DE00080910D028B2917C041E0C41206C080915A
:103DF0000D028B290E94BA11BBCF8091B20582308F
:103E000078F3C812EDCF0E943E0A80910602B812E4
:103E1000B09206028B2D0E949B16AACFC11006C03D
:103E20000E943E0A8B2D0E949416A2CF8091B2056B
:103E300051E0C5120BC0823008F49ACF8091C904BA
:103E40008B2109F495CF0E94640AEACF823040F3B7
:103E5000C812E6CF8DCFDD2029F085E08C1508F45F
:103E600087CFD8CF94E09C1508F482CFDBCFCC204D
:103E7000C9F28091B6059091B705193321F0809170
:103E8000B4059091B5050E946D0C812F0E94A21679
:103E90006FCF802F86958695837069F0813009F009
:103EA00067CF812F902F9370D11002C090E080E0F7
:103EB0000E9427065DCF812F902F9370D11002C0F2
:103EC00090E080E00E943D0653CF812FDD2029F055
:103ED0000E94F2070E9493114BCF0E94D706FACF9F
:103EE000802F837091F5D11043CF412F4295469595
:103EF0004770440F440F812F8F70042E01C0880F2C
:103F00000A94EAF7212F207114FF07C02FE030E058
:103F100001C0220F4A95EAF72095302F3695369545
:103F20003370323069F050F44091AC06313029F0F2
:103F3000822B84230E9452131BCF842B822BFACF17
:103F4000282B8091AC068227F5CF8695DD2011F0D5
:103F5000802F8170882309F40BCF412F429546951D
:103F60004770440F440F812F8F70042E01C0880FBB
:103F70000A94EAF7212F207114FF07C02FE030E0E8
:103F800001C0220F4A95EAF72095302F36953695D5
:103F90003370323069F050F44091AD06313029F081
:103FA000822B84230E94DD12E3CE842B822BFACF56
:103FB000282B8091AD068227F5CFF02FFF70BF2E02
:103FC000DD2029F08F2F0E943113812F24CF812FE4
:103FD0000E9494168B2D0E94EC12CACE123F89F1DA
:103FE00060F4103FB9F0113F81F0DD2009F48CC07E
:103FF000C11060CE802F8F7128C0133F49F1143F4C
:10400000A1F78091790682FF2FC0802F8F71DD206C
:1040100011F31BC0DD2081F024E02C1508F4A8CE9C
:10402000202F2F7181E090E001C0880F2A95EAF7D8
:104030009091AD068927B6CF35E03C1508F498CEAF
:10404000EFCF802F8F71D110C6CF0E94311390CE49
:1040500080E0DD2009F4A6CF81E0902F9F7101C0A0
:10406000880F9A95EAF79ECF8091B2058230A0F131
:1040700080910602DD20F1F00E94500A8091090231
:104080008770843041F40E945D0A802F8F710E94F6
:10409000EC12A12C6DCE8091B205C816D0F7402F3E
:1040A0004F71B42E842F0E94311363E08B2D0E9438
:1040B0003C13EFCF0E94570A8091B205C81640F01A
:1040C0000E945D0A0E94640A64E0802F8F71EFCF26
:1040D00081E00E94F812DDCFDD2059F0502F5F7192
:1040E000B52E852F0E94311363E08B2D0E943C1367
:1040F0003FCE81E00E94F81281E08C1508F038CEA6
:1041000082E00E94F81234CEC110B3CE802F8F719E
:1041100062CFDD2019F0C11038CE3BCEC11035CEB4
:1041200020E0F701408151816281738184810E9486
:10413000590D8091B30583FF28CE8091B1019091F4
:10414000B201029709F021CE812F0E945E171DCE89
:104150000031BFE51B0709F4E1C90131EFE51E0796
:1041600009F4E6C9680127E5D21A882309F4E2C9EF
:104170003FEFC316D10409F008F40ECA8091B105CF
:1041800080FF39C00E9487116C01D70112968C9173
:10419000882309F47ECA8091210182FF08C021E1B1
:1041A00032E040E0B60190E080E00E94B9180B31A7
:1041B000BCE51B0709F45FCA0C31ECE51E0709F4E6
:1041C00060CA90912101892F8E7F90FF81600A3112
:1041D000FCE51F0709F458CAC8019056811520E272
:1041E000920728F0905E8115904108F060CA109205
:1041F000ED041092EC04033FBCE51B0709F4A7CBC8
:1042000008F045CB083DFCE51F0709F49ACB093DB2
:104210002CE5120709F4B3CB073D3CE5130709F081
:1042200042CB06E221EE41EE67ED7CE5C7010E943C
:104230007F17E2C806311C4509F0C1CB8091C90443
:10424000982F9A7A2091B00520FF04C0482F44741B
:1042500009F090E021FF04C0482F417109F090E07F
:1042600022FF04C0482F487809F090E023FF03C0E4
:10427000827209F090E0332309F4BDCC81E0911102
:1042800001C080E08093B00169E2911165E380E9AB
:1042900091E00E94F2050E94E811AEC8CF92DF9231
:1042A000EF92FF920F931F93CF93DF938091C10101
:1042B000807F31F48091BE01C091050281110BC055
:1042C000DF91CF911F910F91FF90EF90DF90CF90F2
:1042D00008952196C7708091C4018C1789F3F090DE
:1042E000BC01E090BD01C090BF01D090C001A6010B
:1042F0006E2D8F2D0E945F06D0E08111EACF8E01D6
:1043000083E0000F111F8A95E1F7F801EB53FE4F90
:1043100081818E11DECF80818F11DBCF828181116F
:10432000D8CFE380F480EC18FD0860E08CEB91E0DE
:104330000E94820D8091AE059091AF05E816F906B6
:1043400040F68091C1018F7080618093C101F801B6
:10435000E653FE4F80818F70806180838CEB91E00B
:104360000E947519DF91CF911F910F91FF90EF90EF
:10437000DF90CF900C948A0A3F924F925F926F9297
:104380007F928F929F92AF92BF92CF92DF92EF92E5
:10439000FF920F931F93CF93DF93CDB7DEB765974F
:1043A0000FB6F894DEBF0FBECDBF8C0185E0F801DB
:1043B000DE01519601900D928A95E1F7D8014C905B
:1043C00011965C9011971296EC9012971396CD90DF
:1043D000DC9060E08CEB91E00E94820D8CEBA82ECB
:1043E00081E0B82E8090BF019090C001A40160913F
:1043F000BD018091BC010E945F068111CAC1F0908D
:10440000BE01F601E819F9094F0160E0FF2009F447
:104410006DC1C5010E94820D6090AE057090AF0520
:104420003090C1018614970408F013C14091BF0178
:104430005091C001B090BC01A090BD01832D807F40
:104440006A2D09F0ADC08B2D0E945F06FE2C8111F4
:104450003BC0D80111968C9111978A1135C08C916F
:104460008B1132C02091C2013091C30116968D91FB
:104470009C912817390741F5E11026C0832D8F70D4
:1044800080618093C1018CEB91E00E94751980914D
:10449000C101F80185838F2D65960FB6F894DEBFB4
:1044A0000FBECDBFDF91CF911F910F91FF90EF9085
:1044B000DF90CF90BF90AF909F908F907F906F9044
:1044C0005F904F903F900895F4EF6F16F1E07F06F4
:1044D00020F48091B30580FF21C0A601652D842DB5
:1044E0000E945F06811118C081E08E2580FF16C0F2
:1044F0004E2D652D842D0E946A0A882379F08CEB5D
:1045000091E00E94751988E0ECEBF1E0DF011D926B
:104510008A95E9F7F12CBFCF80E0E8CFA601652DA1
:10452000842D0E945F06811124C081E08E25B82F62
:10453000B170CB2E80FF2BC04E2D652D842D0E9497
:104540006A0AD82E811123C0498A5A8A89899A8990
:104550000E943F0D292F22952F70223060F02430C9
:1045600088F49F7061F0F8019581907F41F4FD2CF3
:1045700092CF80E0DCCF9F7011F08823C1F3805E82
:104580008830A8F3C8010E947519DC2CF0CFEE200A
:1045900009F481CF8091C10181608093C101BACFBC
:1045A0008B2D0E945F06811124C0D80111968C9139
:1045B00011978A111EC08C918B111BC02091C201D2
:1045C0003091C30116968D919C9117972817390742
:1045D00081F4E1100EC015963C92C8010E94751935
:1045E00088E0F801ACEBB1E001900D928A95E1F71B
:1045F00052CFC8010E944B0D882339F1EE2029F1DA
:104600008091C1018032A0F02091BC013091BD01A8
:104610003A8729871B86DD86CC868E878091C201EA
:104620009091C301988B8F87CE0109960E947519CE
:1046300088E0F801ACEBB1E001900D928A95E1F7CA
:104640000E944E21FF24F39426CFC8010E947519C1
:10465000F9CF832D807F09F452CF9090BC018090D8
:10466000BD014091BF015091C001682D892D0E946C
:104670005F0681111CC0F8018181881118C08081FA
:10468000891115C02091C2013091C30186819781A3
:104690002817390761F4E1100AC03582C8010E9469
:1046A000751988E0D5011D928A95E9F7F4CEC80105
:1046B0000E944B0D882349F2EE2039F28091C1010E
:1046C000803208F4B5CF2091BC013091BD013A830E
:1046D00029831B82DD82CC828E838091C2019091DE
:1046E000C30198878F83CE010196A0CF8CEB91E018
:1046F0000E94820D8091AE059091AF0588169906B3
:1047000080F6FE2CEE2009F4A0CFE090BC01D09002
:10471000BD014091BF015091C0016D2D8E2D0E94B1
:104720005F06811128C0F80181818D1124C080812C
:104730008E1121C02091C2013091C30186819781E1
:1047400028173907C1F48091B30582FD49CF9091B4
:10475000C10190FD45CF907F09F442CF8091C10106
:104760008583903F09F439CF982F907F905F8F70A9
:10477000892B858332CFC8010E944B0D811158CF00
:104780008091C10181608093C101C8010E947519A7
:1047900082CEEE2009F459CFC8010E944B0DF82EAD
:1047A000882309F452CF88E0F801ACEBB1E0019026
:1047B0000D928A95E1F78091BC019091BD010E9414
:1047C0003F0D0E944E2167CECF93DF93CDB7DEB76A
:1047D00060970FB6F894DEBF0FBECDBF29873A872A
:1047E0004B875C876D877E878F87988BCE01099674
:1047F0000E94BC2181112FC088E0FE013996DE01A4
:10480000119601900D928A95E1F74C855D856A8538
:1048100089850E945F0681111EC0A091C401B0E08D
:10482000CD01019687709927209105022817190656
:1048300009F193E0AA0FBB1F9A95E1F7AB53BE4F66
:1048400098E0FE01319601900D929A95E1F78093E0
:10485000C4010E948A0A809105029091C4018913C3
:1048600017C060960FB6F894DEBF0FBECDBFDF91C4
:10487000CF9108950E9456131092C4011092050220
:1048800088E0ECEBF1E0DF011D928A95E9F7E3CFD8
:10489000B8E08B9FC00111248B539E4F0E94BC2116
:1048A0008823F9F28091050290E00196877099279C
:1048B00080930502D0CFEF92FF920F931F93CF9377
:1048C000DF938091F104882361F0C091F0048CE0C3
:1048D000F82E8091F104C81758F01092F10410924C
:1048E000F004DF91CF911F910F91FF90EF90089509
:1048F000EE24E394EC0EE092F0040C2F10E0CF9D38
:10490000E0011124CE50DB4F4B815C8169818881AD
:104910000E945F0681111BC08E819F81892B21F42B
:1049200088859985019651F4288139814A815B8176
:104930006C817D818E819F810E94E423F09EF00135
:10494000F19EF00D1124EE50FB4F14821382CE2DF8
:10495000C0CF10929505109294051092220180917B
:104960009305809392050E9498060C945B243F92D5
:104970004F925F926F927F928F929F92AF92BF926F
:10498000CF92DF92EF92FF920F931F93CF93DF931B
:10499000C091920597E0892E01E010E02CE0322EC4
:1049A0003EEF932E44244394809193058C1315C0BD
:1049B0000E945B24DF91CF911F910F91FF90EF90A8
:1049C000DF90CF90BF90AF909F908F907F906F902F
:1049D0005F904F903F900C949806D0E0FE01EE0F50
:1049E000FF1FE657FA4F80819181889ED001899EF2
:1049F000B00D1124AE5ABA4F14962C911497211170
:104A000057C05090F104E2EFF4E030E020E0712C68
:104A10005D01251508F04AC0E284F384D501CD90EC
:104A2000DC906FEF7FEF612C462D50E0DA01AA0F8A
:104A3000BB1FAC0DBD1D0D90BC91A02D109731F08A
:104A4000EA16FB0609F4BA016394EECF6F3F7607CE
:104A5000A1F1D80102C0AA0FBB1F6A95E2F77A2A1A
:104A6000B80102C0660F771F6A94E2F7AB014150AC
:104A7000510974161506F9F4329EF001339EF00DBB
:104A80001124EE50FB4F889ED001899EB00D112459
:104A9000AE5ABA4F12962D913C91139737832683C5
:104AA000908291829187808715964C920E946A0627
:104AB0002196C37079CF148213822F5F3F4F3C96AB
:104AC000A8CF9F92AF92BF92CF92DF92EF92FF92C8
:104AD0000F931F93CF93DF9300D00F92CDB7DEB724
:104AE00019821A821B828DE5E82E81E0F82E10E0F3
:104AF00000E0CC24C394D12C26E6A22E21E0B22ED5
:104B0000F70181917F018F3F09F445C0F894E82FA8
:104B1000E295EF70F0E021A18F70A60102C0440F72
:104B2000551F8A95E2F7CA01922F982B91A392A163
:104B30008095892382A3789400C0E0E6F1E0912C6F
:104B400031E021912F3F09F465C0A22FA295AF70EB
:104B5000B0E090968C9190E02F7002C0959587956B
:104B60002A95E2F780FD56C0832F982A330FAE16A0
:104B7000BF0639F7F701319780818F3F11F00E940E
:104B80005C0850EA5A95F1F7E1E0F0E0EC0FFD1F08
:104B9000E00FF11F90820F5F1F4F0330110509F0E6
:104BA000AFCF43E050E0BE016F5F7F4F89E192E0FD
:104BB0000E94DD33DD24D394009709F4D12C892B96
:104BC00059F189819A81AB818093190290931A02DD
:104BD000A0931B0281E0809310020E9487119093A2
:104BE0000F0280930E0280910E0290910F020E949C
:104BF00078110597A8F08091190280934D04809157
:104C00001A0280934E0480911B0280934F041092ED
:104C1000100206C080E0A9CF809110028111E3CF7D
:104C2000809100019091010110E006E1019609F0E8
:104C300065C08091220181116BC08091B10580FF18
:104C40001EC08091210182FF1AC00E94871120910D
:104C5000EA043091EB04AC01421B530B20911F017D
:104C6000309120014217530750F021E132E041E03A
:104C7000BC018091EC049091ED040E94B9188D2D37
:104C80000F900F900F90DF91CF911F910F91FF9098
:104C9000EF90DF90CF90BF90AF909F900895089FC6
:104CA000F001099FF00D1124E354FA4FE288F388D4
:104CB000E114F10421F4E090AE05F090AF05089FF7
:104CC000F001099FF00D1124E354FA4F86818823E7
:104CD000A1F0858596850E947811E816F90668F49A
:104CE000109F70011124C70183549A4F0E948112B2
:104CF000C7018D539A4F0E943C121F5F812F90E095
:104D000020910001309101012817390744F691CF15
:104D10008091940590919505009709F48ECF0E949B
:104D200078112091EE043091EF042817390708F02C
:104D300084CF9091920580919305981759F00E9425
:104D4000B7241092EF041092EE0410929505109281
:104D5000940573CF0E945B241092950510929405E0
:104D60000E9498066ACF2F923F924F925F926F9265
:104D70007F928F929F92AF92BF92CF92DF92EF92EB
:104D8000FF920F931F93CF93DF93CDB7DEB7699751
:104D90000FB6F894DEBF0FBECDBF942F498B252FE1
:104DA0005A8B6B8B7C8B8D8B4C895D89622F892F05
:104DB0000E945F06811109C08091B1019091B201FA
:104DC00001969093B2018093B1018B898111109269
:104DD000AE061D861E861F86188A85E0FE01719626
:104DE000DE01199601900D928A95E1F7809179067E
:104DF00082FD1EC08091980590919905892BC1F084
:104E00000E9487112091070230910802821B930BA8
:104E100020919805309199058217930720F0809191
:104E2000090282FFF5C10E94CE1181110E943E0A43
:104E30004C855D856A8589850E945F06811111C058
:104E400061E0CE0109960E94820D6C018B8527EFEF
:104E5000C2162CE5D20681F4882321F181E08093EB
:104E6000220129853A854B855C856D857E858F85F8
:104E700098890E94E423C5C038EFC3163CE5D306E9
:104E800029F4882379F00E94A924EBCF49EFC416B6
:104E90004CE5D40639F4882329F080912201811150
:104EA000F2CFDCCF02E515E0512CB12CA12C22244D
:104EB0002394312C2EEF422EF80140815181882419
:104EC0008A94982C20E0822F90E0FC01EE0FFF1FC7
:104ED000E40FF51F608171816115710531F0C6160F
:104EE000D70609F44C012F5FEECFF12CFFEF8F16A0
:104EF0009F0609F448C0F8014481F09022018F2DEB
:104F0000411180E0F82FF170FF2EF801E5808681D5
:104F10009B85992309F40CC1FF2009F409C1609015
:104F2000AC057090AD05E11012C0A10101C0440FA5
:104F30008A94EAF7842B86838091EE049091EF04A3
:104F40008615970520F47092EF046092EE04C1017B
:104F500002C0880F991F2A95E2F70197F801268170
:104F60002817190681F48091940590919505009772
:104F700009F460C00E9478116816790608F05AC0DA
:104F800021E0F80124835F28FFEFAF1ABF0A095F11
:104F90001F4F28E0A216B10409F08ECF8B8588231D
:104FA00009F421C1552009F41EC10E948711909374
:104FB0009505809394058091F104883010F591E077
:104FC000980F9093F10498E0FE013996DE01119656
:104FD00001900D929A95E1F73CE0839FC001112466
:104FE0008E509B4F28E0FE013196DC0101900D921E
:104FF0002A95E1F72FEF3FEFFC0131872087D38619
:10500000C28669960FB6F894DEBF0FBECDBFDF91A2
:10501000CF911F910F91FF90EF90DF90CF90BF90B5
:10502000AF909F908F907F906F905F904F903F9048
:105030002F9008958091920550919305982FF0E05C
:10504000E0E0851314C090939205E017F10709F48E
:105050009ACF90E0FC01EE0FFF1FE657FA4FB182A6
:10506000A082019683709927809393058CCF682E38
:10507000712CF301EE0FFF1FE657FA4F20813181AB
:1050800047E0429FD001439FB00D1124AE5ABA4F62
:105090006D917C911197798F688F40E020E030E02E
:1050A000E32FF0E0EE0FFF1F688D798DE60FF71FFD
:1050B0008080918081149104E1F0F8010190F081E9
:1050C000E02DFF8BEE8B20E005C08616970609F4D5
:1050D0004F2D2F5FE22FF0E0EE0FFF1F6E897F89CB
:1050E000E60FF71F608171816115710571F73F5FF0
:1050F000D7CF4423D1F0F801231708F0FD0121E0B8
:1051000024830E171F0721F490939205F42E3BCFB2
:10511000981305C0AE17BF0711F49F5F93709301FA
:105120002F5F3F4F822F83708CCFF0E0E0E0F7CF0E
:1051300090E0E1101FC0B10102C0660F771F2A95F1
:10514000E2F79B01215031098217930731F4442380
:1051500009F447C0C5010E946A06C10101C0880F59
:105160008A94EAF7982F9095F8018681892386839F
:10517000FE2C09CF9C01082C02C0359527950A9476
:10518000E2F7A90141705527BC01615071098623DE
:105190009723892B11F5452B01F1F8018281938129
:1051A000892BC1F01B821C821D821E8249824A8289
:1051B0000E9487118160582F9D838C83F801828122
:1051C00093818F83988729813A814B816D817E817C
:1051D0000E94E423F8011582C0CFF22FF170EF2E68
:1051E000BCCFEF2CBACF9091920580919305981780
:1051F00031F00E94B724552009F433CE02CF0E942B
:105200005B2410929505109294050E949806F3CFA6
:1052100082E00E94F81207CECF93DF9300D000D037
:105220000F92CDB7DEB79093C0048093BF04811571
:1052300020E2920748F40F900F900F900F900F907C
:10524000DF91CF910C94D4168EEF89838A831B82D1
:105250000E9487118160782F9D838C8349815A81B8
:105260006B818D810F900F900F900F900F90DF91B9
:10527000CF910C94B3260F931F93CF93DF938C01A0
:10528000EB0165E674E08C2F0E944E0F892BA1F490
:105290008091B4059091B5050E946D0CDD27C35A2D
:1052A000DB4F8881F80110821882833009F148F4BD
:1052B000813059F0823081F0DF91CF911F910F91B1
:1052C00008958430D1F08530B9F7809165049091CC
:1052D0006604009789F306C0809167049091680482
:1052E000009799F3DF91CF911F910F910C940C29A6
:1052F0008091690490916A04F3CF80916B0490913E
:105300006C04009779F720916504309166048091D0
:1053100067049091680421153105D9F2009711F7BF
:10532000C901E0CFCF93DF9300D000D00F92CDB76B
:10533000DEB79093C0048093BF04811520E29207EA
:1053400048F40F900F900F900F900F90DF91CF9136
:105350000C948E188EEF89838A8381E08B830E9460
:1053600087118160782F9D838C8349815A816B815D
:105370008D810F900F900F900F900F90DF91CF9134
:105380000C94B326BF92CF92DF92EF92FF920F93CD
:105390001F93CF93DF93B82EC090AD068091AC06DB
:1053A000C82AC7E0D0E0D12CF12CE12CD701C601EE
:1053B0000C2E04C0B695A795979587950A94D2F7B9
:1053C00080FF1FC04B2D60E08C2F0E949C0C8C0135
:1053D00081309105B1F00E9492298FE39CE90197F9
:1053E000F1F700C00000C8010E940C2981E0DF91A4
:1053F000CF911F910F91FF90EF90DF90CF90BF90D2
:105400000895219798F64B2D60E080E00E949C0C57
:10541000EC010E9492298FE39CE90197F1F700C00B
:105420000000CE01E1CFCF93DF93EC010E949229DF
:105430008091B4059091B5050E946D0CCE01DF916D
:10544000CF910C940C290F931F93CF93DF938C0172
:10545000862F65E674E00E944E0F892BC9F4C09137
:105460006504D0916604209799F0F801808183301B
:1054700069F4CE010E94132ACE010E94132ACE01A4
:10548000DF91CF911F910F910C94132A8430B8F7BC
:10549000DF91CF911F910F9108950F931F93CF9399
:1054A000DF938C01EB0165E674E08C2F0E944E0FB8
:1054B000892B09F064C0FE01FF27D8018C91E35AC3
:1054C000FB4F8130D9F419969C911997992311F0CB
:1054D00080830CC01A969C919923D1F382E080833B
:1054E00080916704909168040097D9F480916504D5
:1054F00090916604009709F442C013C08230E9F528
:1055000019968C91199781112DC01A968C91811141
:105510000EC083E080838091690490916A040097B3
:1055200019F1DF91CF911F910F910C94922984E092
:10553000808380916B0490916C04009791F7809127
:105540006504909166040097F9F00E94132A8091F7
:10555000670490916804009721F780916504909109
:105560006604DFCF85E080838091650490916604B6
:10557000009729F00E94132AF0CF86E08083DF9104
:10558000CF911F910F9108958091670490916804C5
:10559000B1CF1F921FB61F9211248F939F93AF9389
:1055A000BF9380917306811113C08091740690910E
:1055B0007506A0917606B09177064196A11DB11DA2
:1055C0008093740690937506A0937606B093770641
:1055D000BF91AF919F918F911F901FBE1F90189503
:1055E000CDB7DEB7EC970FB6F894DEBF0FBECDBFD8
:1055F00084B7877F84BF0FB6F894A8958091600028
:10560000886180936000109260000FBE80E890E097
:105610000FB6F89480936100909361000FBE85B738
:10562000806885BF85B7806885BF8AE598E09093DC
:105630008F0180938E010E94620F0E94B80F0E941A
:10564000770C0E942E040E94F9048091E20084608D
:105650008093E20078948091A2068823A1F01091B3
:10566000E9001F709091EC00892F817090FD80E817
:10567000182B1092E9008091E80083FD0E946B13C3
:105680001F701093E90082E084BD93E095BD9AEF0E
:1056900097BD80936E000E94900D811102C00E9400
:1056A0003F0F86EC0E945C0887EF0E945C0887E64B
:1056B0000E945C0800E611E086E6E82E81E0F82E04
:1056C000D8018D918D018F3F11F00E945C08E0168A
:1056D000F106B1F783E0EDE4F4E0DF01282F1D923D
:1056E0002A95E9F7E9E1F2E0DF011D928A95E9F7F1
:1056F00090E080E00E9412348A3E9E4F21F40E9486
:10570000900D811102C00E94111082E090E00E9471
:105710000A34809347040E94A90D909379068093E0
:1057200078060E946125EFE3FCE93197F1F700C0AC
:1057300000000E94612580914D0480FF08C06FEF3A
:105740007FEF90E080E00E9436340E94490C83E0B5
:1057500090E00E940A340E94521382E08093420437
:1057600080E880931F020E9498326DE070E08DE81F
:1057700092E00E94430B892BE9F58091420463E09B
:1057800070E081FD28C28AE892E00E94430B892BD9
:1057900089F56DE070E08AE792E00E94430B892B67
:1057A00049F50E94BC05605A75418F4F9F4F609329
:1057B000C3047093C4048093C5049093C604E2E4C8
:1057C000F2E080E092E0DF019C011D922150304028
:1057D000E1F7F0932102E09320028FEF9FEF909387
:1057E00045048093440481E08093C8048093C704F7
:1057F0001092430422982A9A23982B9A83B182FB11
:10580000882780F91B99EAC190E0892B80931E02BA
:1058100082E091E09093700680936F064424439455
:10582000512CBE016F5F7F4F7B011E0173E0270E7D
:10583000311C8091A20610E102E1853009F41EC2FC
:105840000E946125A82E81110E94BC05ADE4B4E040
:10585000E8E4F4E010E000E0302F8D91919198178A
:1058600009F41BC2292F282790E0DD24D394422F6E
:105870004D2109F40DC29BA73CA78D2191E009F4AD
:1058800090E09DA70E9487118160782F9FA78EA727
:105890004BA55CA56DA58FA50E94B326F801E85B1A
:1058A000FB4F8081D826D082E0911E02EE0FEE0FD2
:1058B000E0931E0283B182FB882780F98DAB1EAA7C
:1058C0001B9902C280E02DA93EA9822BE82BE09310
:1058D0001E02EF70F0E0EA59FE4F808190911D02A8
:1058E000890F80931D02B12C823054F080911C02EC
:1058F0008F5F80931C0280E00E94C229BB24B39476
:1059000080911D028F3F54F480911C02815080933E
:105910001C0281E00E94C229BB24B39480911D0225
:10592000082E000C990B62E070E00E94B333809364
:105930001D02B1100E94BC058091C804882309F49F
:10594000A5C082E492E090932102809320022091EE
:10595000440430914504DC0190E080E0FC01E6560F
:10596000FD4F64914D916417A1F0AD014150510973
:10597000FA016083AC0115E0569547951A95E1F759
:10598000B20102C0660F771F4A95E2F7AB01262BE2
:10599000352B0196811572E0970701F73093450486
:1059A000209344042115310509F457C08091430424
:1059B000811153C0082F10E06201082E02C0CC0CE8
:1059C000DD1C0A94E2F7A60142235323452B09F478
:1059D0007EC19091420490FD7CC18295880F8076B3
:1059E0008093100198013695279536952795209339
:1059F0001301815E809311011092140124E630E0BE
:105A000047E050E06EE071E088E70E944733892B61
:105A100021F5A801F5E0440F551FFA95E1F78091B3
:105A2000420480FD64C14E5B5D4F04E610E020E25D
:105A300030E060E488E70E946E33892B71F40E94A5
:105A40008E0BC094D0948091440490914504C82258
:105A5000D922D0924504C09244048091C70488237F
:105A6000A9F00E94BC050091C3041091C4042091C8
:105A7000C5043091C604601B710B820B930B6F3F02
:105A80007F4F8F4F9F4710F40E94730BA11001C0EE
:105A9000B1100E948E0B86E0E7E5F4E0D70101909B
:105AA0000D928A95E1F7C0905904D0905A04009164
:105AB0005B0410915C041092590410925A041092E5
:105AC0005B0410925C048C2D8D2991F0809155041B
:105AD000909156040E947811AC0190915104992341
:105AE00009F46EC180911D018417150608F476C172
:105AF000802F812B91F080915304909154040E9447
:105B00007811AC0190915004992309F4A6C18091B9
:105B100019018417150608F4AEC1809159049091BB
:105B20005A04892B90915B04892B90915C04892BFA
:105B300011F00E94931186E0F701A7E5B4E001900F
:105B40000D928A95E1F70E945306909146048917B9
:105B500021F00E945306809346048091A20684306F
:105B600009F067CE83E08093E9008091E80082FF2E
:105B700060CE8091E80090E085FF09C00E944D044E
:105B800000E210E06701882309F4BDC191E0809133
:105B9000E8008B778093E800992309F44ACE0091BE
:105BA000C1041091C20489810115110509F4B9C11C
:105BB0008E3F09F0F8C18A81833020F08550833010
:105BC00008F0F1C1EA81EE3008F0EDC1F0E0E658EE
:105BD000FB4C0C94C73387E892E0D7CD92E015CE0A
:105BE0008091A206843031F10E94730B10927306EB
:105BF00088E190E0A0E40FB6F894A8958093600047
:105C00000FBEA093600083B7817F846083BF83B79A
:105C1000816083BF7894889583B78E7F83BF0FB6EA
:105C2000F894A8958091600088618093600010923C
:105C300060000FBE8091A106882301F10E946125BA
:105C400080914E0490914D04892B90914F04892BA3
:105C5000A9F019BD09BD09B400FEFDCF8091D8009F
:105C60008F7D8093D8008091E00082608093E00077
:105C70008091E00081FDFCCF0E9456138091A20626
:105C8000853009F4ADCF0E9456130E945306D8CD3B
:105C90009F5FDD0C963009F0EACD0F5F1F4F033098
:105CA000110509F0D9CD8FEF88AB89AB1AAA0E94F4
:105CB00087118160782F9CAB8BAB48A959A96AA941
:105CC0008CA90E94B326F0CD82E090E0FCCD8F5FDE
:105CD00071CE880F880F880F8093100110921301E6
:105CE000895F8093110183E08093140187CEE2E203
:105CF000F2E080E2DF011D928A95E9F7EAE7F1E040
:105D0000FCAFEBAF66E771E0E7E08E2EEBADFCADEC
:105D1000A191FCAFEBAFFB018191BF01840F952FE7
:105D2000911D9C012E5B3D4F3AAF29AFEA2FF0E069
:105D3000EE5DFD4F90E080E0682C681A942C082EF0
:105D400001C0990C0A94EAF7A9ADBAADB8AFAFABF0
:105D500000E0AFA9B8AD1D91B8AFAFAB1921262DAA
:105D6000201B2770722E022E000C330BB12F01C0A6
:105D7000BB0F7A94EAF77B2E319521953109277074
:105D8000332701C016952A95EAF7712A1081712AE6
:105D900070820F5F0830E9F60196319688309105E0
:105DA00059F6EEE7F1E02BAD3CADE217F30709F051
:105DB000ADCF04E610E020E230E042E252E039CE1E
:105DC00020911E016AE0269F9001112424173507B7
:105DD00008F08ECE9F5F9093510402C09F3FD1F791
:105DE000CC2059F00E9493079FEF1C140CF491E013
:105DF000899F802D112480935904DD2059F00E9441
:105E000093079FEF1D140CF491E0899F802D1124BE
:105E100080935A0430915904332309F469CE2091B8
:105E20005A04222309F464CE75EB3703C001112410
:105E3000992359F09093590445EB240390011124C0
:105E4000332339F030935A0453CE81E080935904C0
:105E5000F3CF81E080935A044BCE20911A016AE07F
:105E6000269F900111242417350708F056CE9F5F16
:105E70009093500402C09F3FD1F7002359F00E9435
:105E80005A079FEF10160CF491E0899F802D112482
:105E900080935B04112359F00E945A079FEF11165B
:105EA0000CF491E0899F802D112480935C04309143
:105EB0005B04332309F431CE20915C04222309F4DE
:105EC0002CCE75EB3703C0011124992359F0909320
:105ED0005B0445EB240390011124332339F0309304
:105EE0005C041BCE81E080935B04F3CF81E0809360
:105EF0005C0413CE8091F100D6018D936D010150A9
:105F0000110909F443CE8091E80085FDF3CF80911B
:105F1000E8008B778093E8000E944D04882399F372
:105F200035CE8D3009F49DC0B0F4843009F480C0C2
:105F300040F4823041F108F06CC0813001F18FEF04
:105F4000CCC2863009F48AC008F47DC08C30B9F721
:105F500080E18A8328C0813109F4DCC040F48F30AD
:105F600009F4ACC008F481C00E94140E1CC0833137
:105F700009F4F9C008F4D0C08E3F09F723CE1A8285
:105F800089E08B8310C08A81823009F4C8C28330D3
:105F900081F18130A1F60E94BC050E94CD336B8354
:105FA0007C838D839E838091A206843009F041CC4E
:105FB0008091E9008F702091EC00122F117020FD6C
:105FC00010E8182B82E08093E9008091E80080FFC0
:105FD0000CC050E040E060E270E0C7010E947E0427
:105FE0009091E8009E779093E8001F701093E9006D
:105FF00020CC8091150190911601892BA1F28091FE
:106000004D048B8380914E048C8380914F048D834B
:10601000CACF8A81823009F092CF6B817C818D81D9
:106020009E810E94CD3386E290E00E941834BBCF5F
:106030004C816B818A810E94C50C982789279827FB
:106040009E838D83B0CF2D813E8132272327322737
:106050004C816B818A810E94550EA5CF0E94A20EB1
:10606000A2CF82E08A8387E78CCF0C8110E00D31CC
:10607000110508F098CFCA80DB80DC24CD24DC2415
:1060800057010E0D1F1DC60187579E4FA016B10662
:1060900009F489CFB7E7CB16B2E0DB0658F40E94CB
:1060A0000A34F5018483BFEFCB1ADB0AEFEFAE1A97
:1060B000BE0AE9CFD50114961C92F5CF8091150147
:1060C00090911601892B09F46ECFCC80D12CFDE183
:1060D000CF16D10408F067CF0A811B811027012752
:1060E00010275701C00ED11EC80187579E4FC016FA
:1060F000D10609F458CF073722E0120728F4D5015A
:1061000014966C910E941834BFEFAB1ABB0A0F5F54
:106110001F4FEACF84E01DCF0C8110E00D31110537
:1061200008F041CFCA80DB80DC24CD24DC24570179
:106130000E0D1F1DC6018796A016B10609F433CFB8
:10614000E0E9CE16D10460F40E940A34D501149619
:106150008C93FFEFCF1ADF0A2FEFA21AB20AEACF11
:10616000F5011482F6CFCC80D12C3DE1C316D104C9
:1061700008F019CF0A811B81102701271027003949
:10618000110508F010CF80E990E0801B910B8C1571
:106190009D0508F408CF5701C00ED11EC80187968F
:1061A0000C151D0509F4FFCE0039110528F4D501A1
:1061B00014966C910E941834BFEFAB1ABB0A0F5FA4
:1061C0001F4FECCF88E0E4E2F1E0DE019196019010
:1061D0000D928A95E1F780E2F70111928A95E9F72D
:1061E00084E0898388E0FE01B196DE011596019076
:1061F0000D928A95E1F7D7CE84E3898381E08A8383
:106200001B821C82D0CE8C81682F70E0762F66278F
:106210008B81860F972F911D092E000CAA0BBB0BAB
:1062200035E0880F991FAA1FBB1F3A95D1F7AC0123
:10623000BD01405E5F4F6F4F7F4F481759076A0798
:106240007B0708F4B0CE8433F1E09F07A105B105C8
:1062500008F0A9CE453321E052076105710520F011
:1062600044E351E060E070E0481B590BBC01665606
:106270007B4FC7010E94D43396CE1B810C8140E036
:10628000602F812F0E949C0C9827892798279A833A
:10629000898341E0602F812F0E949C0C98278927D9
:1062A00098279C838B837FCE2E813F8132272327A3
:1062B00032274D816C818B810E94240E74CE4EE179
:1062C00050E06FEF70E0C1010E94F333809115013F
:1062D00089830A8368CE61E070E07093C2046093A2
:1062E000C10482E390E090934C0480934B040E949D
:1062F000871159CE8091150189830A8380914B04BF
:1063000040CE0B811C8140E250E06FEF70E0C7018E
:106310000E94F3332EE536E090E080E0AC014E5F62
:106320005F4F4132510508F03ECEF90165917491FD
:106330000617170730F48E0D9F1DDC016D937C93BB
:10634000CA01285F3F4FB6E0263F3B0739F72BCE07
:106350002B813C818EE596E0FC01459154914217DA
:10636000530709F4A4C00896E6E0863F9E07A1F70C
:10637000E6CD8B819C810EE516E0F80125913491E4
:106380008217930709F4ABC0085F1F4FF6E0063F82
:106390001F0799F7D4CD0E94D30D05CE8B81823093
:1063A00009F449C0E0F48823F1F1813009F0FBCD14
:1063B0008C819AE0D92E8E010F5D1F4FF8012D2D93
:1063C00011922A95E9F7B8010E944E0F8983F801CE
:1063D000DE01129601900D92DA94E1F7E4CD83305C
:1063E00009F447C0843009F0DECD6C818AE0FE01FB
:1063F0003596DE01919601900D928A95E1F78FEF27
:10640000683068F4FAE06F9FB0011124675C7E4F3A
:106410004AE050E0CE0181960E943C3480E08983BE
:106420000E94B80FC0CD8EE1D1011D928A95E9F787
:1064300088E089838ECD6C818AE0FE013596DE018D
:10644000919601900D928A95E1F78FEF683068F48C
:106450003AE0639FB001112467517F4F4AE050E05A
:10646000CE0181960E943C3480E089830E94620FB5
:106470009ACD6C812AE0CE018196DC01E22F1D923B
:10648000EA95E9F7683088F4629FB0011124675CEF
:106490007E4F4AE050E00E94FA3380E089838AE030
:1064A000FE01B196DE011296A2CE8FEFF7CF9C01CE
:1064B0002E5F3F4FF901459154914032510508F04C
:1064C0003ECDF90145915491FC013496659174914A
:1064D000CE0102960E94EA3380E0898364CDC80130
:1064E0000296FC01259134912D31310508F027CD1C
:1064F000FC0145915491F801349685919491BE0127
:106500006B5F7F4F0E94EA330E94B70DF801369609
:1065100085919491009701F3FC010995DDCF86E206
:1065200090E00E940A341B821C821D828E833BCD28
:106530001092B9008CE08093B80008959F92AF92BA
:10654000BF92CF92DF92EF92FF920F931F93CF9360
:10655000DF93B82EEB010E9487116C01EE24E394C7
:10656000F12CC431D10560F025E0E22EF12CCF3FB3
:10657000DC0731F0CE0164E170E00E949F337B01C3
:1065800084EAA82E94E8992E1092BC00A092BC0038
:106590000E9487118C018091BC0087FF0DC0809103
:1065A000B900887F883039F18091B900887F8031C7
:1065B00011F10FEF1FEF09C00E948711801B910B93
:1065C0008E159F0540F30EEF1FEFCF3FDC07E1F282
:1065D000C6010E9478118C179D07B0F2C801DF91A7
:1065E000CF911F910F91FF90EF90DF90CF90BF90D0
:1065F000AF909F900895B092BB009092BC000E9413
:1066000087118C018091BC0087FF0AC08091B9007E
:10661000887F883111F0803461F610E000E0DECF31
:106620000E948711801B910B8E159F0558F3CBCFCD
:106630000F931F93CF93DF93EB018093BB0084E80C
:106640008093BC000E9487118C018091BC0087FF61
:1066500011C02091B900287F81E090E0283211F428
:1066600090E080E0919581959109DF91CF911F9104
:106670000F910895CF3FDC0741F30E948711801BE3
:10668000910B8C179D0708F38EEF9FEFEECFCF9203
:10669000DF92EF92FF920F931F93CF93DF936B01E3
:1066A0008A017901B9010E949E32E6010C0D1D1D7F
:1066B000C017D10761F424E92093BC00DF91CF918A
:1066C0001F910F91FF90EF90DF90CF90089597FD6D
:1066D000F2CFB70189910E941833EACFCF92DF92AF
:1066E000EF92FF920F931F93CF93DF93C62F6A0110
:1066F0007901B8010E949E3297FD0CC0B8018C2F21
:106700000E941833E601EC0CFD1CCE15DF0511F0DC
:1067100097FF0CC024E92093BC00DF91CF911F911B
:106720000F91FF90EF90DF90CF900895B80189917D
:106730000E941833EACF84E98093BC000895AA1B15
:10674000BB1B51E107C0AA1FBB1FA617B70710F05C
:10675000A61BB70B881F991F5A95A9F7809590958E
:10676000BC01CD01089597FB072E16F4009407D0C5
:1067700077FD09D00E949F3307FC05D03EF4909529
:1067800081959F4F0895709561957F4F0895EE0F05
:10679000FF1F0590F491E02D09946927962769273A
:1067A0007827872778270895FB01DC0102C0059030
:1067B0000D9241505040D8F70895FB01DC0104C010
:1067C0008D910190801921F441505040C8F7881BE9
:1067D000990B0895FB01DC0102C001900D9241501C
:1067E0005040D8F70895DC0101C06D9341505040EE
:1067F000E0F70895DC01CB01FC01F999FECF06C05A
:10680000F2BDE1BDF89A319600B40D92415050406E
:10681000B8F70895F999FECF92BD81BDF89A9927EE
:1068200080B50895A8E1B0E042E050E00C94FC335C
:10683000262FF999FECF92BD81BDF89A019700B439
:10684000021639F01FBA20BD0FB6F894FA9AF99AD9
:106850000FBE08950396272F0E9419340E94183402
:10686000252F0E941934242F0C9419340196272FB8
:106870000E9419340C941834DC01CB0103C02D9113
:106880000E94473441505040D0F70895262FF9997F
:10689000FECF1FBA92BD81BD20BD0FB6F894FA9A03
:1068A000F99A0FBE01960895F894FFCFFE0AFE0AEA
:1068B000070B070B090B070B070B070BFE0AFE0A5A
:1068C0000E0B070B070B0E0B5114791427167914B6
:1068D0002716AC14CD142716D615E315421E421EFA
:1068E000781E781E491F651FB81EB81E701FDD1F59
:1068F000EE1FEE1FE230FC3003313D3154315F3189
:106900006B317A31D32F8131A831B931CB31CE31CE
:10691000FFFFB905090CE80BE40BE00BB8050021FB
:10692000007F22000301002808641E140A321EAFF3
:10693000000101018DA31A095BD6A232818283E294
:1069400000E900EA00B500B600B700CD008301CC35
:10695000008A0192019401210223022402250226C9
:106960000227022A02B300B4006F007000C6F76766
:10697000F0F1F4F5F63700FF0100010000FFFF0021
:1069800000010001FF000008101818100800402244
:0E699000BC8A016801AC000C07250745070012
:00000001FF
